:100000006F4080291300000013000000130000005F
:100010001300000013000000130000001300000094
:100020001300000013000000130000001300000084
:08003000130000007300100032
:1000380000000000000000002E0400003204000050
:1000480000000000DE410000000000000000000089
:10005800E0410000E2410000000000000000000054
:100068000C400000000000005C02000000000000DE
:10007800E8410000EA410000EC410000EE410000C8
:10008800F0410000F2410000F4410000F641000098
:10009800F8410000FA410000FC410000FE41000068
:1000A8000042000002420000044200000642000034
:1000B800084200000A4200000C4200000E42000004
:1000C80010420000124200001442000016420000D4
:1000D800184200001A4200001C4200001E420000A4
:1000E8002042000022420000244200002642000074
:1000F800284200002A4200002C4200002E42000044
:100108003042000032420000344200003642000013
:10011800384200003A4200003C4200003E420000E3
:1001280040420000424200004442000046420000B3
:10013800484200004A4200004C4200004E42000083
:100148005042000052420000544200005642000053
:10015800584200005A4200005C4200005E42000023
:1001680060420000624200006442000066420000F3
:10017800684200006A4200006C4200006E420000C3
:100188007042000072420000744200007642000093
:10019800784200007A4200007C4200007E42000063
:1001A8008042000082420000844200008642000033
:1001B800884200008A4200008C4200008E42000003
:1001C80090420000924200009442000096420000D3
:1001D8000000000000000000000000000000000017
:1001E8000000000000000000000000000000000007
:0801F8000000000000000000FF
:1002000083A2418503A1020011A0010082427390E4
:100210001234924273900230A240B2414242D24222
:100220006243F243025492542255B2554256D2567A
:100230006257F257064896482649B649464AD64A72
:10024000664BF64B065C965C265DB65D465ED65EFA
:10025000665FF65F0961730020300100197116CAEC
:100260009302000273A04280F322003016C2F322F0
:10027000103416C006C40EC612C81ACC1ECE22D028
:1002800026D22AD42ED632D836DA3ADC3EDEC2C0A6
:10029000C6C2CAC4CEC6D2C8D6CADACCDECEE2D076
:1002A000E6D2EAD4EED6F2D8F6DAFADCFEDE8A82BC
:1002B00003A1018216C0EF30304E02419382418586
:1002C0001383018683A3020023A0230003230300DA
:1002D00023A0620003210300924273900230824205
:1002E00073901234A240B2414242D2426243F2437E
:1002F000025492542255B2554256D2566257F25782
:10030000064896482649B649464AD64A664BF64BB1
:10031000065C965C265DB65D465ED65E665FF65F01
:10032000096173002030397101436EC619A039711B
:1003300041536AC866CA62CC5ECE19A039710153B6
:100340005AD056D252D44ED64AD826DA22DC06DE0D
:1003500033016140828241114AC026C222C406C6CE
:100360008282B24D4101024D924C224CB24B41016E
:10037000024B924A224AB249410102499244224424
:10038000B240410182803D432A876373C302937761
:10039000F700BDEFADE5937606FF3D8ABA960CC334
:1003A0004CC30CC74CC74107E36BD7FE11E28280F8
:1003B000B306C3408A069702000096966780A6009F
:1003C0002307B700A306B7002306B700A305B700AD
:1003D0002305B700A304B7002304B700A303B700A5
:1003E0002303B700A302B7002302B700A301B7009D
:1003F0002301B700A300B7002300B700828093F564
:10040000F50F93968500D58D93960501D58D61B72F
:10041000939627009702000096968682E78086FAD8
:100420009680C1171D8F3E96E374C3F8A5B773007D
:10043000203001A0EFF23FF237C400001305040B97
:10044000EF70E06A81451305007DEF30D00DFDB7F8
:10045000EFF2FFEDB7C4000037C90000AA8A2E8B67
:10046000328A01449384C40A1309496DB7CB000052
:10047000634844012945EF708056EF10A050E5B560
:10048000A68911C0CA8993173400DA978C43D043E8
:1004900056850504EF1000142A86CE8513854B047B
:1004A000EF70C04FF1B7EFF27FE9375500209305A9
:1004B000007D13058534EF1000482A84EF10604D4D
:1004C0002A893705000013050545AE89EF10004C59
:1004D000B7C600002A87AE879386060CCA854E866B
:1004E0002285EF10804BB7C500009385850C2285CF
:1004F000EF106055B7C400009385440D2285EF10BE
:10050000805481451305803EEF30F001F5B7EFF2DE
:100510009FE4716513050520EF40600DB7070020CB
:1005200083A5071E37C500001305C504EF700047FB
:10053000B7C5000037C500009385C50513054506FE
:10054000EF70C045EF30A04F0D64B70700203706AD
:100550000000B7C50000373500208148130804802B
:10056000938787250D4781461306464393854508A3
:10057000130585A5EF30E04EB737002037060000A1
:10058000B7C50000373500208148130804809387E1
:1005900087B4114781461306664A9385C50813053B
:1005A00005ADEF30004CEF30C03B37C50000130500
:1005B0004509EF70C0530100FDBFB71702409843D3
:1005C000B706FFF841111367170098C3D8433706E1
:1005D0000200758FD8C39843B706F7FEFD16758FD6
:1005E00098C39843B706FCFFFD16758F98C3D84390
:1005F000B70681FFFD16758FD8C39843B70600EC88
:10060000FD16758F98C33707FF0098C723A607020A
:1006100002C402C69843C166558F98C3B7160240FC
:1006200005679C42F18F3EC6A24785073EC4B2478C
:1006300081E7A247E397E7FEB71702409C43139771
:10064000E7006357070685473EC632478547631F65
:10065000F704B7170240D843B706C1FFFD16D8C349
:10066000D843D8C3D84313670740D8C3D843758F3E
:10067000D8C3D843B7061D00558FD8C39843B706D3
:100680000001558F98C3984393166700E3DD06FE7B
:10069000D843B7160240719BD8C3D84313672700CD
:1006A000D8C32147DC42B18BE39EE7FE4101828043
:1006B00002C661BF13D745019307F07F1545631547
:1006C000F700C18113F5F5008280EFF2DFC8DD3756
:1006D00059151335150055B138517C4D411102C6DD
:1006E0006374F700998F3EC6B247584163F3E70041
:1006F0005CC17C5578006377F700998F184163736C
:10070000F7001CC141018280AA8701456308B50238
:100710006307D5003307A6000307070001E785C17B
:10072000AA8501A83388A7002300E8000505F9BFC2
:100730007D153E95230005002E85828075F9828007
:10074000130E0002914E9306F0021303A002294FEC
:100750006364B600328582803307C5000308070052
:1007600093071600630CC803930878FF93F8F80FFB
:1007700063F61E0363F8B7026316D802B308F500E8
:10078000838808006390D802930726006388B70027
:100790003307F500030707006314E7013E864DBFEA
:1007A0008507EDB793083600E3F6B8FAE314D8FAF4
:1007B000AA9783870700E39F67F893074600E38FB4
:1007C000B7FC030627006316660003063700E3073D
:1007D000D6FC85070507E5B7639BB600EFF2BFB708
:1007E000B2853686EF50D0711335150079B60145C4
:1007F0008280AA87130505FD1375F50F2547637DD4
:10080000A7001387F7F91377F70F954663E7E6001C
:10081000938797FA13F5F70F82801387F7FB137707
:10082000F70F0145E3EAE6FE938797FCE5B71377F8
:1008300035008546AA87630ED700214501CF89463A
:100840007D556319D70013D527000D057199110542
:10085000828041458280EFF21FB041112A84AE842C
:1008600032C6A53501C5324600C244C2410131B687
:10087000EFF27FAE38517C4D411102C663F0E702C2
:10088000B7C6000037C500009386863413860183FF
:100890009305E0091305C535EF5090603C4D1146B6
:1008A0006800BE95EF50306832454101F9B4EFF26F
:1008B0009FAA41112E8436C6653FB24609817D1537
:1008C00088C21305440041014DBCEFF2DFA82C495A
:1008D0002A849105713FB707F07F28C87CC871BC96
:1008E000EFF27FA72A892E842E85B285B284D93370
:1008F00019476315E5003335800041B41547AA87D1
:10090000631BE500014681462285A685EF40106203
:100910003335A000DDB70545EDD31D47E38FE7FC78
:1009200009470145E39BE7FCA2854A859137098188
:100930007D15F9BFEFF29FA0AA84B6893A8A0D3FD0
:10094000BC501374C5FF637AF40219E022850DB41C
:10095000930544002685293FAA852A892685093FD3
:10096000B04C935625001109FD164A96D2854E8546
:10097000A53569FDA2852685D9B70144C1BFEFF22F
:10098000FF9B41112A892E84B28485492285A68540
:100990001533631D35018325890521042146A29560
:1009A0002800EF5050582244B244CDB72285A68586
:1009B00041017DBA830705001307F005638BE70645
:1009C000130740026387E70693F7F7FD9387F7FB6A
:1009D00093F7F70F6547637EF70481473E85828072
:1009E000850404C2044263F6B402B307950083870A
:1009F0000700E38707FFE38517FF13F7F7FD1307EA
:100A0000F7FB1377F70FE37DE3FC938707FDE3F92B
:100A1000F6FC1C215D479387E7F993F7F70F636AAC
:100A2000F73431678A071307070FBA979C432A8464
:100A30008287EFF25F921308F00593084002654346
:100A4000A5464DB72A8637C50000A68695451305ED
:100A5000053A5933894719C1930720033E856FF042
:100A6000DF912A8637C50000A68695451305853A8D
:100A7000A533930750037DF137C50000A686228673
:100A800091451305053B893B9307300361F937C551
:100A90000000A686228695451305853B353B9307C6
:100AA00040034DFD37C50000A686228695451305F7
:100AB000053C1D339307600355F137C50000A6863A
:100AC0002286A1451305853C013B894741D99307FF
:100AD000700369B72A8637C50000A68689451305C5
:100AE000453DDD399307A00335F937C50000A686DB
:100AF00022869D451305853DC531894725D193073C
:100B00008003A9BF2A8637C50000A6869145130534
:100B1000053ED931894739D19307B00381B72A8679
:100B200037C50000A6868D451305853E75319307B0
:100B3000D003E31505F237C50000A6862286A1453D
:100B40001305052251399307E003E31905F037C572
:100B50000000A68622869D451305C53EB53993073C
:100B6000C003E31D05EE37C50000A6862286954525
:100B70001305453F95318947E30205EE93071005BC
:100B8000F1BD2A8637C50000A68689451305C53FF5
:100B9000A1319307F003E31305EC37C50000A686E7
:100BA0002286894513050540053993070004E3179C
:100BB00005EA37C50000A6862286A94513054540EB
:100BC00021398947E30C05E89307100441BD2A86C3
:100BD00037C50000A6868D4513050541F53E8947BA
:100BE000E30E05E69307200495BD2A8637C500006D
:100BF000A6868D4513054541C53693073004E31F8E
:100C000005E437C50000A6862286914513050547F1
:100C1000E1368947E30405E49307F00481B52A86A9
:100C200037C50000A6869945130585417536894765
:100C3000E30605E29307400415B52A8637C5000090
:100C4000A686994513050542413E8947E30805E01C
:100C50009307500421B52A8637C50000A6868D4526
:100C600013058542953E93078004E31905DE37C5D9
:100C70000000A686228691451305C542B13E930722
:100C80006004E31D05DC37C50000A6862286954575
:100C900013054543913693077004E31105DC37C50E
:100CA0000000A686228691451305C5433536930775
:100CB0000005E31505DA37C50000A68622869945AA
:100CC00013054544113E8947E30A05D89307A0065A
:100CD00071B32A8637C50000A686A545130585474A
:100CE000E53C8947E30C05D69307E00485BB2A86DB
:100CF00037C50000A6868D451305C544F13C930712
:100D00009004E31D05D437C50000A68622869145D0
:100D100013050545D1348947E30205D49307A004A0
:100D200035BB2A8637C50000A6869545130585453F
:100D300065349307B004E31305D237C50000A686D7
:100D40002286914513050546413C8947E30805D0B5
:100D50009307C00421B32A8637C50000A6869545AF
:100D600013058546953C8947E30A05CE9307D004D1
:100D7000F5B18947E5B1EFF20FDE0329050304451C
:100D800050592A8423070502A30605024111CA858A
:100D90002685EFF0FF9A48D808DC232E0402636909
:100DA00025018547A306F402054541016FF0EFDCFC
:100DB000AA94838704001307F0026384E720634941
:100DC000F708130780026382E7146340F7041307F0
:100DD00050026387E7206343F7021307100263831F
:100DE000E71413072002638EE72EB305A94013060C
:100DF000C4032685C136A306A402F5A81307600222
:100E0000638FE71E13077002F9BF1307B002638CEC
:100E1000E7166346F70213079002638AE70E13078B
:100E2000A002E394E7FC0505637A25198387140083
:100E30001307A002639DE7169307D0063DA2130790
:100E4000D002638BE710635CF70C9307400645A064
:100E50001307E0036383E7246342F7041307A00347
:100E60006382E70A63CDE72C1307C0036386E71E9E
:100E70006355F70A9307150063FD271D8387140048
:100E80001307D0036397E71C09056374251D0387C7
:100E900024006310F71C9307A00745A81307B007A9
:100EA0006389E7066346F7021307F003638FE702DF
:100EB0001307E005E39BE7F205056371252303872C
:100EC00014009307D003631BF7209307D0F871A891
:100ED0001307D0076381E70463C7E7141307E0072C
:100EE000E395E7F09307900619A0930720F8A3066F
:100EF000F40285475CDC1C5C585C0345D402BA975D
:100F00005CD865B5930710F8DDB79947CDB79D4715
:100F1000F9BFA147E9BFA547D9BF9547C9BF930707
:100F2000F0F8F1B79307150063F527030387140062
:100F30009307D003631FF7000905637C250103872E
:100F400024006318F7009307B007A306F4028D4747
:100F500055B79307800661BF0505637325030387B3
:100F600014006318F70093077006A306F40289477C
:100F700051B79307D0036315F700930750F8F5B7FF
:100F800093072007ADB70505637025030387140099
:100F90006315F70093076006C9BF9307D003631575
:100FA000F700930740F8D1B79307100789B71307E5
:100FB000D0036395E700930760F845BF9307E00609
:100FC0003DB70505637B2501038714009307D00314
:100FD0006315F700930770F849BF9307F00601BF48
:100FE0000505637B2501038714009307D003631570
:100FF000F700930780F895BF93070007CDBD05055F
:1010000063702503038714006315F7009307F00747
:10101000A9BF9307D0036315F7009307C0F8B1B7D2
:101020009307C007E9B5050563722503838714009C
:101030001307C0076395E700930700F83DB7130750
:10104000D0036395E7009307E0F805B79307E0073F
:1010500079BD930730F861BD13071500637C270342
:10106000038714006311F7020905637B25010387D9
:1010700024009307D0036315F700930790F8F1B5A8
:1010800093073007DDB59307D0036315F700930787
:101090007007E1BD9307600799BD13071500637CD6
:1010A0002703038714006311F7020905637B2501F9
:1010B000038724009307D0036315F7009307A0F874
:1010C00069B59307400755B59307D0036315F7003B
:1010D0009307900759BD9307800711BD9307D00769
:1010E00039B585475CDC9308C005130380075C5C59
:1010F000838504003388F4003307F50003060800F5
:10110000637C27036397C5001147A306E4028507A4
:10111000D5B38546631F160193062700636ED90079
:101120000308180089466316680011076366E90022
:101130009146B6975CDC65BFE31FB6DAF1B726854A
:101140006C00EF70B0038D47A306F402B24728C4C9
:101150006CC4B384974044DC79BB0347E50201E7E4
:101160000345D5028280EFF20F9F31316FF0EFA07F
:10117000EFF2CF9C41112A84AE89EFF06FEF2A89FC
:1011800063580502284CB704008093C7F4FFB37777
:10119000F9002C0011464E953EC4EF50C05893C53F
:1011A000C4FF93773900B375B90081EF2285C93741
:1011B000370500801345C5FF3375A90041016FF065
:1011C0002F9B0547E396E7FE22855D37938549000F
:1011D0002285EFF0EFE9AA852285593F2C4CA10921
:1011E0002146CE952800EF500054A244B2452685F2
:1011F000EFF04FCC894763F5A7009D47E31AF5FA56
:10120000A6856DB7EFF22F920111AA892E8A2E853D
:10121000B285B6843A8932C6EFF0CFC9A547AA860F
:1012200063E9A71E31679317250013070715BA97BF
:101230009C433246828737C60000A5461306864780
:10124000CA852685EFF04FCC05616FF08F9137C6C8
:101250000000914613060647E5B7137A1A00631893
:101260000A0037C600001306463F9546D1BF37C671
:1012700000001306C6439146E1B737C60000854615
:101280001306064DCA852685EFF00FC82A84D2853D
:101290004E85EFF0EFDD137BC5FFB7CB000037CCF9
:1012A000000083A70906B38C8400330D8940637462
:1012B000FB00631D0B0037C6000085461306C64DB4
:1012C000EA856685EFF04FC42295BDBF93054B00BC
:1012D0004E85EFF0EFD983A5890593078B00AA8D82
:1012E000BE9521462808EF5000449306F4FFB3361C
:1012F000D00013864B4DEA856685624AF24AEFF0CC
:10130000AFC02A9433078940B3868400EE85370640
:10131000F27F4E85C53D2A94B30589408546130664
:101320008C4D33858400EFF02FBE2A94330789401B
:10133000B3868400D28556864E85E935DA852A94AF
:101340004E85EFF0EFD2137BC5FFA1BFD2853408E5
:101350004E85EFF0CFD537CA0000AA8A854613061E
:101360000A4ECA852685EFF02FBA03A68905E24604
:101370002A845696B305A9402695EFF0EFB82A9433
:10138000854613060A4EB3058940338584001DBF88
:10139000B287B28952853008BE85EF60007601467B
:1013A00081465289EF40803819C9B7C5000093853E
:1013B000C54C4A86CE862685EF60700671B5B7C5E6
:1013C00000009385454CF5B7D28534084E85EFF083
:1013D0000FCE37C600002A8AA14613060622CA8508
:1013E0002685EFF06FB203A689052A84E24652965D
:1013F00059BF37C60000D2861306464ECA852685D9
:10140000EF60E07A91B537C60000D2861306464FEA
:10141000F5B737C6000013060650CDB7397126CA96
:1014200032D49304C50037C6000022CC4AC82A84AF
:101430002E8936D61306062E9D4693051002268564
:1014400006CE3EDA3AD842DC46DEEFF0EFAB93054B
:1014500010023410898D4A86269536C6EF70606F6B
:101460001C5823070402F2405CD8930700105EB4B6
:101470006244D24442490145B705FA7F2161828026
:10148000EFE2DFEB205193877600784D4111F19B1D
:101490002EC6A297AA84637BF700B7C50000938588
:1014A00005382685A53F41016FE09FEC3CD1FD57F3
:1014B000E305F4FE284DB2896C0011462295368969
:1014C000EF506026638A0900BC4C130544004A862D
:1014D000CE853E95EF508030B24589478D89639720
:1014E000F500BC4CA297CA97A3810700C205B707B5
:1014F000F07F2285DD8D45BFEFE2FFE5204D79715C
:10150000AA842E94A2851146680842C636C23EC4FB
:10151000EF506021A24792460C103ED4B2471146CC
:1015200022853ED6BC5036D23ED0EF50C01FF24589
:101530005010B146F199268593E515009137456124
:101540006FE0BFE3EFE23FE18347F5024111858B96
:1015500099CFB7C6000037C500009386463813867A
:1015600081839305D0221305C535EF5060133C49A4
:101570007000914681452A843EC6193728C86CC838
:1015800041016FE09FDFEFE21FDD41112EC62A848B
:10159000B284E136B245630EB500B7C5000093854D
:1015A000C5292285A53D88C0CCC0014541016FE019
:1015B000DFDC85472307F4020545CDBFEFE2BFD945
:1015C00093061600939726002E8693E527004D3D3F
:1015D0006FE0BFDAEFE29FD6AA842E892E85B2850E
:1015E000B289EFF08F8E1384C4000DE5B850FC4C27
:1015F0009306470063F3F602A04CF117CA853694B0
:101600004E863387E740A2862685ED3E2A868145B1
:1016100026856D3722856FE0BFD537C400001304DF
:10162000C40ACDBFEFE23FD01C5D83298500244D65
:101630000111BE993C5113874700BA94585DBA977F
:10164000784D91076371F710B7C500009385053891
:10165000F13305616FE0FFD0338529010821631B59
:10166000750D4E97182303C509006313A702B387AE
:10167000C40098A305090506CA87485C138727009C
:1016800013891700E36AA7FC22858145053FD1B77E
:1016900063178701B387C40023800701E1BF631686
:1016A0009701B387C4008CA3F1B76316A701B38772
:1016B000C40094A3C1B76319B707138937003387F0
:1016C00029010823130705FD63FAEA001377F5FDE6
:1016D0001307F7FB1377F70F6368EB04CE97D82354
:1016E000930707FD63FAFA009377F7FD9387F7FBFB
:1016F00093F7F70F636AFB0242CE2ECC36CA32C88C
:101700003AC6EFF00F8F32472A8A120A3A85EFF075
:101710004F8E4246336AAA00D246B387C400238064
:101720004701E2457248B9B7B7C500009385453215
:10173000228539BF1C44185CCA97BA979823B3878F
:10174000C40098A30DBF2A8401468147930BC005AE
:10175000130CE006930C4007130D2007930D800730
:10176000A54A154BB546A545294801BFEFE2BFBBC9
:1017700041112A84EFE05FF63840FD576307F71404
:101780008144B70900803C5063EBF4022448A685ED
:101790002285EFF0FF9D938544002285EFF04F8D69
:1017A000AA8475F52C4081C52285EFF07F9CB70A8D
:1017B0000080814493CAFAFF054B894B21A2A6857C
:1017C0002285EFF0EF8A2A89284CB3673901114648
:1017D0002C0026953EC4EF4010754A85EFF02F850A
:1017E000AA9455B7A6852285EFF08F88AA8933750C
:1017F0005501EFF0CF832A8963D5090C014A370CD4
:10180000F07F9D4C95A0D2852285EFF06F86AA8946
:1018100033755501EFF0AF812A8D63C6090493F744
:101820002900B1E363FB3401284CB38729411146F9
:101830002C0052953EC4EF40106F93F93900639924
:10184000090893094A00CE852285EFF06F8263FC78
:10185000A4003C4C330525412AC411462C00338595
:101860003701EF40506C6A9A3050E36ECAF83C483A
:1018700063F8F400B38727413CC8B707F07F7CC802
:101880003C4063E59700B38727413CC01C44284C8B
:10189000637CF500744C3387A7406377D70063F50A
:1018A000E400B38727411CC4B38524010D8EAA959B
:1018B0002695EF40B0723C503389274123202407FE
:1018C0000149CA943C50E3EFF4F041016FE07FA975
:1018D000E39B69F993094A00CE852285EFE05FF921
:1018E00063FCA4003C4C330525412AC411462C005E
:1018F00033853701EF4030633C4C930D8A0021461D
:10190000BE9DEE852800EF401062A249B2454E858B
:10191000EFE05FDA63F4AB00E31795F5E3F534F538
:1019200042053365AC00B38929412AC64EC421461D
:101930002C006E853DB7EFE21FA29307700741119F
:10194000014463FDB7022E86AE8481452A84EFE010
:101950009FA393070407938404F93CCC64CC91467D
:1019600070008145228502C6EFF09FB17C4C28C8EB
:101970006CC8E19B7CCC5CC085837CD02285410116
:101980006FE0BF9F0145B705F37F8280B705F97F00
:1019900082800145B705F07F8280EFE23F9A2A847A
:1019A0002E892E85B285B289B6843A8ABE8AEFE046
:1019B0007FD00DE12685EF60E02A2A86A685228564
:1019C000F53EAA862E87D2875688CA854E862285FE
:1019D000EFF09FB26FE0DF99EFE25F9601110147F0
:1019E000B707F37F3ACC3ECE1307F6FFF5572A84AC
:1019F00063F8E7002E852EC6EF60C026B2452A8622
:101A000085472307F4023C08A30604020CC410D83F
:101A1000232A04027CD485442285EFF00FF4624926
:101A2000F249630795004A85CE85EFE01FCA11C5CC
:101A30004A85CE8505616FE0BF932285EF0090391E
:101A40002ACC2ECED1BFEFE21F917D5671376FE0C9
:101A5000DF92EFE25F8DBE8C8347F5021D71858BAF
:101A6000639D0778B28AAE89B28536863A8C2A8D14
:101A7000368BEFE0DFF02A84AE846686E2856A85E5
:101A8000EFE0FFEF2A896A852E8AEFE0FFC4228506
:101A9000A685EFE09FC32DED4A85D285EFE0FFC21A
:101AA000631105769387D90793F7F70F2D47636383
:101AB000F7765685DA85EFE0FFBF8547630AF5764E
:101AC000B7C50000938505206A85EFF03F953DA8D6
:101AD000D2854A85EFE01FBEB1652A841306000354
:101AE000938545010818EF401044AD4763E787022E
:101AF0000A049C103E94832504FD2E852EC0EF60C1
:101B0000601682452A866A85EFF05FAB2A84AE8430
:101B10002285A68525616FE0DF84B7C50000938527
:101B2000C51FE1BF4A85D285EFE0DFB8A147630753
:101B3000F500B7C500009385852079B72285A68575
:101B4000EFE05FB7930795FF93F7D70FAA8A91C786
:101B5000B7C500009385452185BFB70500018329DE
:101B60008D00FD153375B900220A135989018327A9
:101B70004D0333692A01B375B9004E95832B0D03CC
:101B80002324AD002328BD0201463EC0EFE05FBB29
:101B90008347DD02232AAD0201493EC28347FD028D
:101BA0003EC483270D043EC69D47638BFA049D44C3
:101BB000130AF008854A03274D0383270D03636842
:101BC000F71E83258D058327CD0513561940131A5B
:101BD0003900BE950E06AE86338545012E966115F9
:101BE000631AD6224A866A8502942A846A85AE845C
:101BF000EFE09FAE8327CD05D297232EFD04A5AA43
:101C0000A285268674106A85EFE07FCA83248D053D
:101C10009307C5FF2320FD04AA946A853254054B1F
:101C2000EFF05F92130A9002094C854CB70DF37FD9
:101C3000930AC00263788B0E5A86A2852685EFE050
:101C40003FB02A8B3389A40063768500830709009F
:101C5000638747151018B30564414A8502D8EFE041
:101C60007FD5631F850B83278D0003264D038325B6
:101C70000D033E853EC8EFE0BFACC247232AAD024C
:101C800023079D03AA97038707006E888147630790
:101C900047016A85EF00E07AAA872E8803230D05A5
:101CA00083234D054256CA856A8542CE3ECC1AC86A
:101CB0001ECAEFF0BF904243D243E2477248AA8661
:101CC0002E871E869A856A85EFF01F8383270D0372
:101CD00003298D0003264D03BE854A853EC8EFE0EB
:101CE0003FA6C247232AAD02637AF5002A998307EB
:101CF0000900639557010505232AAD024256A285C6
:101D000026855A96EFE0DFA32A8BE37585F2B38729
:101D1000A40083870700E39F57F1130B150019BF39
:101D2000636F8B065A86A2852685EFE07FA1637BD1
:101D30008500B387A400038707009307B0076313E8
:101D4000F700050591471306F4FFB385A400098E3B
:101D5000A307FD026A8549312A84AE84EFE0FF962D
:101D600001E98347FD02C18B81E70144B704F37F9A
:101D70006A85EFE09FB5824723243D0123287D0338
:101D8000232AFD02A247A307FD029247A306FD02F4
:101D9000B2472320FD0485472307FD0295BB0307B7
:101DA000090093079002E31FF7F6050BA5BF6A85AC
:101DB000EFF0AFBAE30795E06A85EF0080682E8602
:101DC000AA856A85EFE0BFBB03270D068327CD05F3
:101DD0002AD82EDA210763FCE700B7C500009385F7
:101DE000C5226A85EFF08FE32A84AE8469B70325A4
:101DF0008D05E117232EFD0421460C183E95EF407A
:101E000090126A850509EFF04FB5E31645DB23070D
:101E10005D0355B318415C4103A3060083A346004C
:101E200098C2DCC22320650023227500A10645BBB1
:101E30000147B707F03F5686DA86930540086A8562
:101E4000EF106057F1B10147B707F03F5686DA86C9
:101E500093055008EDB74A85D285EFE0BF859947D5
:101E60006310F50213341900B704F67F55B14A87A1
:101E7000D2875686DA86CE856A85EF10C05379B14F
:101E80002285A685EFE01F838947AA8A631FF50C88
:101E90004A85D285EFE01F822A8B6318550D3410D6
:101EA000A28526866A85EFE09FA05286AA8A7410D2
:101EB000CA856A85EFE0BF9F930710072A8A639956
:101EC000F9042256B25781456A853E96EFF00FEF2E
:101ED0002A84AE84EFE00FFEE31C65C31418A285CC
:101EE00026866A85EFE0BF9C2A8903258D05225648
:101EF000B30555014A95EF40700EA25703258D0595
:101F000032563E99B30545014A95EF40300D09B16F
:101F10009307A0076391F9022256B2570144E315D3
:101F2000F6F403258D05B30545015695EF40407D38
:101F30001334150015BF9307B0076393F9022256B7
:101F4000B2570145631BF60003258D05B305450116
:101F50005695EF40E07A133515001344150029B764
:101F6000B7C500009385852385B69387A9F993F7B4
:101F7000F70F1947636EF7004A85D285EFE08FF3BC
:101F800095476304F502B7C50000938545242DBE2F
:101F900093074006638BF9009547E396FAFE4A855E
:101FA000D285EFE02FF1E31055FF9387C9F993F73E
:101FB000F70F6947228BA68B6367F72231678A0781
:101FC00013078717BA979C438287014681464A8543
:101FD000D285EF30A07511E5B7C500009385452582
:101FE000E5B44A86D2862285A685EF30E01839BE50
:101FF0004A86D2865A85DE85EF300018EF40004FC2
:10200000EF4040554A86D286EF30300F2A86AE86A2
:102010005A85DE85EF30F059D5BC4A86D2862285B6
:10202000A685EF30900DDDB44A86D2862285A6853E
:10203000EF209021E1BC4A86D286D9BF2285A685B1
:10204000EF40C04A2A84D2854A85EF40204A218D3C
:10205000EF40405065BC2285A685EF4020492A8488
:10206000D2854A85EF408048618DDDB72285A685FF
:10207000EF40C0472A84D2854A85EF402047418DF2
:10208000C1BFB70500804A84B3C4450151B44A8535
:10209000D285EF40A0451345F5FF5DBF014681465F
:1020A0004A85D285EF30806861B52285A685EF40EC
:1020B000E0432A84D2854A85EF4040433315A4008B
:1020C00041BF2285A685EF4060422A84D2854A8599
:1020D000EF40C0413355A440A5BF4A85D285EFE00B
:1020E0006FDDA1476307F500B7C50000938505269E
:1020F000E1BAB707000103258D00FD173377F9001A
:102100003A9509476399EA02220A93558901B36512
:10211000BA0037C60000994613060627FD8DEFE08A
:10212000AFEB01CDA2856A85EFE08FF409817D15C3
:10213000EF404049E1BA63870A00B7C500009385C4
:10214000852759B2220A135789013367EA00AA8604
:102150007D8FA28526866A85EFE0CFFD5DC52A8446
:10216000B704F17F75B22285A685EF4020382A8416
:10217000D2854A85EF408037098C13341400EDB1C5
:102180002285A685EF4080362A84D2854A85EF4095
:10219000E035098C33348000C1B922854A86D28665
:1021A000A685EF30206A132405007DB922854A8672
:1021B000D286A685EF3000691324150075B12285FB
:1021C0004A86D286A685EF30005D3324A00069B927
:1021D00022854A86D286A685EF30E05B1345F5FF5F
:1021E0001354F50151B1B7C500004E866A85938539
:1021F000C528EFF0AFA26FF07F91014481446FF0EA
:102200003F914A84D2846FF0BF900144B704F37FBA
:102210006FF01F909387B9F993F7F70F1547E361B4
:10222000F7C631678A071307471EBA979C43828710
:1022300093073008E39DF9C203258D0593F7CAFF84
:10224000A10721460C183E954AD852DA5684EF4031
:10225000804DDA846FF0DF8BEFE24F8E41112A84DC
:10226000EF10E00E2A89AE849309E007054A4A85FB
:10227000A685EFE08FC511E52285EFE01FEE63082C
:1022800035034A85A685EFE04FC409ED8349F40282
:10229000130AF007854A2285EFE03FEC630345050A
:1022A000A30734034A85A68541016FE06F8C23079D
:1022B00044032285834AD402EF1060092AC62EC443
:1022C000EFE0AFC0A247324711E94A86A686D6851D
:1022D0002285EFF00FF82A89AE8451BF3A89BE8477
:1022E0004DB72686CA85230754032285EFE02FE9E0
:1022F000AE842A89AA8526862285EFE06FDE834791
:10230000F40201E993E71700A307F4022285A93735
:1023100059B7858BE5FF228581372A89AE84A5BF11
:10232000EFE2CF812A840D3F2A89AE89EFE0EFB931
:1023300009ED8344F402130A0008854A2285EFE080
:10234000DFE163084501A30794024A85CE856FE06B
:102350002F824E86CA85230754032285EFE02FE2A1
:10236000AE892A89AA854E862285EFE06FD78347FA
:10237000F40201C993E71700A307F40222854D3741
:1023800075BF858BE5FF2285613F2A89AE897DB7C0
:10239000EFD2DFFA2A84930A2008054A130B1008AB
:1023A0002285BD3F2A892285AE89EFE01FDB6314B9
:1023B00055074E8623074403CA8522858344F402C9
:1023C000EFE0EFDB2E86AA852285EFE06FD121C9F1
:1023D00022857D3F8347F4022A89228593E71700EF
:1023E000A307F402AE89EFE05FD793071008630EEE
:1023F000F500B7C50000A30794029385C52922857F
:10240000EFF0CF812A89AE8939A0230744032285C2
:102410004137A30794024A85CE856FD07FF5834765
:10242000F402228593E71700A307F402953722856B
:10243000EFE0BFD2E31F65FB23074403A307940229
:1024400085B7EFD2BFEF41112A8499372A89AE842C
:1024500093093008294A854A4A85A685EFE0EFA608
:1024600031E52285EFE07FCF630A35018347D4024F
:102470009387C70793F7F70F636AFA02230754039A
:102480002285034BD402753F2AC62EC4EFE0EFA38A
:10249000A247324711E94A86A686DA852285EFF0FF
:1024A0004FDB2A89AE844DBF3A89BE844A85A68512
:1024B00041016FD0FFEBEFD21FE78344F502854760
:1024C0004111AA8B85882307F502054A814C370DF7
:1024D000F37F8549130CF0085E85EFE01FC889473C
:1024E000630AF500B7C500005E859385C529EFE056
:1024F000FFF295A823874B035E8583AD8B0303A969
:10250000CB0303A48B00EFE01F8793073008668B93
:10251000EA8A631BF50023874B035E851D372A8BF0
:10252000AE8AEFE08F9A31E199C85E85EFE0FFC295
:1025300095476314F508014BB70AF37F3DA083A5C7
:102540000B0503A64B056E944A87A2865E85EFE0D5
:102550006FBE0DC1B7C50000A2864A869385852C43
:102560005E85EFE0BFEB2A8BAE8A5A85D6854101A6
:102570006FD03FDF03A30B0583A34B054A86A285DB
:102580005E851AC41EC6EFF06F8356862AC02EC21F
:102590005E85DA85EFE0AFBE2243B2438246124742
:1025A000AA872E881E869A855E85EFE0FFF42A8B27
:1025B000AE8AEFE08F9135D94DBF5E85EFE0FFB970
:1025C000E30B35F75E85EFE05FB9E31D85F1238707
:1025D0003B0319B7EFD23FD538517C5141112A84C2
:1025E00063F4E700EFF08F982285EFE01FB79307C1
:1025F000D0036308F52063E0A7069307600363E157
:10260000A702930730036375F502A1476303F51E24
:1026100093072003630BF5082285EFF09FE2EDA6F8
:102620009307A00363E4A70293078003636DF50497
:1026300014441C5C505CB7C50000BE969385852E83
:102640002285EFE0BFDD2A89AE8451A09307C00345
:10265000E300F5FED1B793072004630AF50A63E9A6
:10266000A7009307F0036308F50AE373F5FC6DB761
:10267000930740046300F534E36CF5FA9307D00444
:10268000E3ECA7F875B78347F40213F7170015EBCF
:1026900013F7270093E717001DE3B7C500009385E4
:1026A00005302285EFE09FD779BF8347F40213F707
:1026B000170001EB13F7270093E7970079DFA307D3
:1026C000F40285472307F4020149B704F37F22850A
:1026D000EFE0BFA89547630FF5322285EFE0FFA733
:1026E00085476309F5322285EFE03FA7A5476303DD
:1026F000F532B7C50000938585312285EFE01FD202
:102700002A89AE844A85A68541016FD09FC522855E
:10271000EFF07FDA0DBF8544230794022285EFE0B6
:102720008FE599476307F500B7C500009385C52974
:102730008DBF230794022285EFF0BFD02E86AA8595
:102740002285EFE0CFA32A892285AE89EFE0FFA0A2
:102750009D47E31BF5FC4E8623079402CA8522851C
:10276000EFE00F988347F402AA8993FA170009E56E
:1027700093E71700A307F40222851D2E2A89AE8451
:10278000639C090063970A008347F402F99BA3073F
:10279000F4020149B704F37F034BD402832B4403B3
:1027A000054A230744032285EFE0EFDC9307B003DB
:1027B000232A7403A3066403E31BF5F023074403F1
:1027C0002285EFE09F99230744036388090083472C
:1027D000F40293E71700A307F4022285D12CE384C7
:1027E00009E6E3960AEE8347F402F99BA307F40295
:1027F000F9BD8345F402228593C5F5FF8589392CFF
:1028000099B58344F4020147B707F37F13F9140025
:102810003AC43EC6631509002285EFE0BFD23000FE
:102820009305D0032285EFE01FD66309050E300023
:1028300099452285EFE03FD56302050E2285EFE042
:10284000DF919547631DF50A300095452285EFE03D
:102850009FD36305050C8347F4022285032A4403B2
:1028600093E71700A307F402EFE03F8F9547631E3D
:10287000F50A300095452285EFE0FFD045C122855D
:10288000832A4403EFE07F8D9D476319F50A3000EA
:102890009D452285EFE03FCF51C12285032B4403A4
:1028A000012C3000EFD03FFB35E9832B44038549F1
:1028B000154C9D4C6310090CA3079402232A440372
:1028C000230734032285EFE00FCB6311850983478B
:1028D000F402232A64032307340393E72700A307A2
:1028E000F4022285F1223000EFD0FFF641CD22859F
:1028F000EFD0BFFDA30794022249B244C9BB228591
:10290000EFE0BF8593072004631DF5002285EFF0FB
:102910009FBA3000EFD03FF4E30805F2E31C09FC56
:10292000F9B72285EFF0FFB1EDB72285EFF07FB167
:102930003000EFD05FF2E30E05F2CDB72285EFF065
:102940005FB03000EFD03FF139D1C9BF2285EFF041
:102950005FAF2E86AA852285EFE06F8230002A8D38
:10296000AE8DEFD05FEF41F5EA856E862285EFD020
:102970003FF731FD9547232A7403A306F40223078A
:10298000040269BF8347F402A18BEDF7A307940209
:10299000232A5403230734032285EFE0CFBDE30D40
:1029A00095F12285EFF0FFA93000EFD0DFEAE305D3
:1029B00005F035BF8349F40285472307F40293F7F6
:1029C000590091E7B7C500009385C530D9B9228574
:1029D000EFE0AFF895470149B704F37FE309F5CE7F
:1029E0002285EFF01FA62E8693F91900AA8522856D
:1029F000EFD0FFF8639A09001C585CD88347F402B3
:102A000093E70701A307F4022E86AA852285EFD05B
:102A10001FF715B985472307F402EDB1EFD23F91B7
:102A20002A842E8A99C1EFE0FFB185472307F4027B
:102A30000149B709F37F854A254BA14B130CF003DD
:102A4000930CB004154D2285EFE02FF16309550575
:102A50002285EFE08FF0630465054A85CE85EFD0CF
:102A6000DFC615ED22858344D402EFF0BFB62A8974
:102A7000AE89EFD09FC561F9E38774FDE38584FDDE
:102A8000E38394FD8347D402E38FA7FBB7C500001F
:102A9000938585312285EFE07F982A89AE89630589
:102AA0000A002285EFD07FE24A85CE856FD0BF8BAA
:102AB000EFD27F8A2A84EFE04FEAA147631CF5003A
:102AC0008345F402228593C5F5FF8589EFF01FF554
:102AD0006FD0BF8A2285EFF0FFAF2E86AA852285B0
:102AE000EFD0FFE923070402E5B7EFD2DF8301113E
:102AF0002A8CEFE08FE699476314F5040549230714
:102B00002C036285EFF0FF932A84AE84EFD0FFBBE5
:102B10001DE16285EFE06FE49D47630CF500B7C5EA
:102B200000009385852A6285EFE05F8F2A84AE845A
:102B300019A023072C032285A68505616FD07F820B
:102B40006285EFE08FE16285EFD01FB983278C06A5
:102B500091CB03270C0063F7E700B7C5000093850E
:102B6000452BD1B78347DC02054423078C0221475C
:102B7000638CE7066367F70209476385E7266368A6
:102B8000F700F5C3B7C500009385C52B69BF0D4796
:102B90006387E7041147E397E7FE6285EFE09FA8AC
:102BA00071B71307F0046380E726636EF70013071D
:102BB000E003638DE7141307E004E395E7FC0144A9
:102BC000B704F37F8DBF130700056382E724130763
:102BD00010050144E398E7FAB704F67FA9BF032480
:102BE0008C048324CC0481BF034AFC02137A1A00AC
:102BF00063100A08914670088145628502CEEFE0B5
:102C00003F882A84AE842285A685EFD01FAC05F5C7
:102C100085472307FC02A54B914C854A130D1008EC
:102C2000930DF0086285EFE04FD3630E750783477D
:102C3000DC0209476392E70481490149631E0A00E7
:102C400083258C0083278C030326CC036285BE95E5
:102C5000EFE0DF96AA892E8923075C036285EFE007
:102C60008F916305A503B7C500009385C52965BD90
:102C70000144B704F37F41BFE39797FF81490149BE
:102C8000E31C0AFC6285EFE0FF99E9B723075C03C8
:102C90006285EFF00FFB2A8B63010A026285EFE089
:102CA000CFCB631D75056285EFE02FCBA547E31CF5
:102CB000F5FA85472307FC02BDBD2EC6EFD0FFA065
:102CC0003246631805144E85CA85EFD01FA005E56E
:102CD0003246DA856285EFD09FCAAA872E88CE86D3
:102CE0004A87A28526866285EFE01F81AA892E8900
:102CF000EFD0BF9D45D54E84CA8435BD6285EFE0D7
:102D0000CFC5E312B5F723075C0329BF62850349EA
:102D1000FC02EFE04F8699476305F500A3072C03FB
:102D200099B783294C0323078C02854A01449D44AB
:102D3000094B054A930BF0086285EFE00FC2630D63
:102D4000550315C46285EFE04FC1E31965FD230704
:102D50004C036285EFE02F82630095026285EFE00D
:102D6000CFBFE31D75FB23074C030544F1B7628514
:102D7000EFE0AFBEE31895FC6285EFE00FBE9D4724
:102D8000E31EF5F8054A23074C036285EFD0BFFE2A
:102D9000A147E315F5F88347FC0223070C028145A0
:102DA00093E71700A307FC026285EFF03FC72A8470
:102DB000AE84EFD09F9101C5A3072C03ADBB0326C2
:102DC0004C0383258C00FD19A3072C0333063641E1
:102DD000CE956285EFE08FFE2A8423074C03B7046B
:102DE000F77F91BB0324CC0383278C039354840087
:102DF00013970401A20762044183A183B704F87FFB
:102E00005D8CD98C0DBB0144B704F47F2DB3054410
:102E1000E1B35A84B28405B3EFD2EFD041112A8CCA
:102E2000EFE0AFB3930780066309F5048347DC0244
:102E3000938777F993F7670FA9C36285EFF0FFCA0D
:102E40002A89AE89EFD07F882DCD4A85CE85EFD0F7
:102E5000DF8725E16285EFE04FB08345DC0205475F
:102E60009387A5F993F7F70F6365F7042307EC023F
:102E7000814701474A86CE8605A80344DC029307B2
:102E80002007630DF402930710076314F400130482
:102E9000B00685472307FC026285BD3FAE872A87BF
:102EA0000146B706F37FA2856285EFE09FBA2A89C3
:102EB000AE894A85CE8541016FD0AFCA1304C006E2
:102EC000C9BF4A85CE85EFD0EFFEA1476313F50455
:102ED0008347FC02858BD9EF370400017D14B3775B
:102EE0008900A20983248C001359890133E929013F
:102EF00003264C0583290C05BE9433748900228770
:102F0000A686CE856285EFD0FFA215CD2A89B709A6
:102F1000F17FC16A370B0001CA844E841D4AFD1A35
:102F20007D1BB7CB00006285EFE02FA399476306B6
:102F3000F5046285EFE06FA293074006630FF50288
:102F40002689A28919B7638B090093854900628598
:102F5000EFD01F92AA893706F07F55B7B7C500009A
:102F6000A6862286938545336285EFE02FCB2A899A
:102F7000AE8945B70149814969BF0347DC02930720
:102F800040066314F70285472307FC026285EFF0D1
:102F9000DFB5AE872A872686A2869305400662851E
:102FA000EFE03FABAA842E84BDBF8349FC02032916
:102FB0004C03854C93E71900A307FC0285472307C0
:102FC000FC02130DF0088147854D62853EC6EFE097
:102FD000CF98B247630B9501A1C76285EFF06FC62A
:102FE0006285EFE08F97631345056285EFE0EF960A
:102FF00063074505A3073C039385CB296285EFE072
:10300000EFC12A89AE894A85CE85EFD00FECE31E49
:1030100005E24A87CE872686A2869305500641B7E9
:103020006285EFE08F93E31A45FBC1B76285EFE05D
:10303000CF92E311A5FD2307BC03854779B703268B
:10304000CC038547A3073C033305C90003264C0383
:1030500033796901B709F87F098E93568600B3F674
:10306000560162062307FC0233692601B3E9D90041
:1030700059BFEFD2AFAC41112A84EFF0FFD92A89B2
:10308000AE849309E006054A854A4A85A685EFD0B5
:10309000CFE339E52285EFE04F8C630A35018347A2
:1030A000D402938717F993F7F70F636BFA0223079C
:1030B00054032285034BD402EFF01FD62AC62EC438
:1030C000EFD0AFE0A247324711E94A86A686DA85FB
:1030D0002285EFE01F982A89AE8445BF3A89BE84D5
:1030E0004A85A68541016FD0AFA8EFD22FA5411127
:1030F0002A89EFF01FF8AA842E84930A1007130A76
:103100002007054B2685A285EFD02FDC11E94A85E3
:10311000EFE0AF848349D902630955016387490110
:103120002685A28541016FD0AFA4230769034A8594
:10313000EFF03FF42AC62EC4EFD02FD9A247324772
:1031400011E92686A286CE854A85EFE09F90AA8463
:103150002E844DBFBA843E84E1B7EFD24F9D41111A
:103160002A84EFF09FF82A89AE84130A4007930A55
:10317000300793095007054B4A85A685EFD0EFD459
:1031800005E12285EFD07FFD630145032285EFD065
:10319000DFFC630C55012285EFD03FFC630735014E
:1031A0004A85A68541016FD00F9C230764032285C1
:1031B000834BD402EFF07FF32AC62EC4EFD0EFD0BA
:1031C000A247324711E94A86A686DE852285EFE0CE
:1031D0005F882A89AE844DB73A89BE84D1B7EFD2D1
:1031E0000F9541112A84EFF05FF72A89AE84130A04
:1031F0006007930A7007130B800793099007854BAC
:103200004A85A685EFD06FCC0DE52285EFD0FFF47F
:10321000630645032285EFD05FF4630155032285E1
:10322000EFD0BFF3630C65012285EFD01FF3630776
:1032300035014A85A68541016FD0EF9223077403BB
:103240002285034CD402EFF05FF12AC62EC4EFD0E2
:10325000CFC7A247324711E94A86A686E285228572
:10326000EFE02FFF2A89AE8461BF3A89BE84D1B7CF
:10327000EFD2CF8C41112A84EFF07FF62A89AE84F9
:10328000130AA0079309B007854A4A85A685EFD09F
:10329000CFC319E92285EFD05FEC630C450122858D
:1032A000EFD0BFEB630735014A85A68541016FD09A
:1032B0002F8C230754032285034BD402EFF03FF2F7
:1032C0002AC62EC4EFD06FC0A247324711E94A8602
:1032D000A686DA852285EFE0CFF72A89AE8475B716
:1032E0003A89BE84D1B7EFD26F8541112A89EFF0B8
:1032F0003FF8AA842E849309C007054A2685A28533
:10330000EFD0AFBC11E54A85EFD03FE5630735014B
:103310002685A28541016FD0AF85230749034A85E1
:10332000834AD902EFF0DFF42AC62EC4EFD0EFB9FA
:10333000A247324711E92686A286D6854A85EFE064
:103340004FF1AA842E845DBFBA843E84D1B7EFC208
:10335000FFFE41112A89EFF01FF9AA842E849309F8
:10336000D007054A2685A285EFD02FB611E54A85FC
:10337000EFD0BFDE630735012685A28541016FC00E
:103380003FFF230749034A85834AD902EFF0BFF57F
:103390002AC62EC4EFD06FB3A247324711E9268662
:1033A000A286D6854A85EFE0CFEAAA842E845DBF47
:1033B000BA843E84D1B7EFC27FF8BE89B7776E6F0B
:1033C0000111938717273ECAB7777475938707371C
:1033D0003ECCE17793C7C7D7FC869307E007230F5E
:1033E000F1001C10BE9583CA05F73284B28536867B
:1033F0002A8AB6843A89EFD08FD8AE864A87CE879C
:103400002A86D6855285EFE0CFE483278A052AC431
:103410001375C4FF21052EC621462C003E95EF30C2
:1034200080302285A68505616FC09FF45C4111053F
:10343000F19B3E958280EFC21FF22A84EFF01FFFBE
:1034400000C16FC09FF3B7670020B76600201387E5
:1034500007D7138606D823A807D6232207002324DC
:1034600007002326070010CF50CF232007021305A3
:103470000706938707D7938606D8130800022322EE
:103480000702BE85014623A2D50805069105E31C67
:1034900006FF110793870708E313A7FE8280417791
:1034A000698FAA871305000219E3C2074145370750
:1034B00000FF7D8F19E3A2076115370700F07D8FAC
:1034C00019E392077115370700C07D8F19E38A074A
:1034D000791563C307007D158280EFC2DFE793078C
:1034E000F00741112A8463EAA700135425400145DF
:1034F00088C100C241016FC05FE832C62EC4EFF040
:103500001FFA9307A5FF3354F440134404026515D2
:103510003246A245F1BFEFC21FE42A84484141115F
:1035200070002C007199EFF05FFBA246B24537673F
:10353000002093975600AE9793870702130707D78B
:103540008A07BA97C84337660020130606D808C40E
:1035500050C440C51053C0C385473395D700A1065A
:10356000498E8A0610D336975443B397B700D58F48
:103570005CC341016FC07FE0EFC25FDC37640020B5
:10358000832604D78D47638AF606130704D781473D
:10359000130904D763CDD704E11513773500F199EA
:1035A0009307003231E337070040938645FF5117F8
:1035B00093071032636AD70293E515009309C5FF9C
:1035C0000CC1AA844E85EFF01FF54E85EFF0BFE6E3
:1035D00089475CC1832704D7138717008A07CA97D6
:1035E000C4C32328E4D681473E856FC07FD8110726
:1035F00010436307C500850771BF93072032EDB7FD
:1036000093073032D5B7EFC21FD541112AC62EC459
:10361000EFF07FE3A2453245EFF01FF641016FC0A6
:10362000DFD5EFC2BFD15C4D184D0449A9495CC339
:1036300098C3232805002306050003C98405630AEF
:103640003901CA852685EF000062238C34056FC0DE
:103650003FD24C2983C714022A84E38AB7FE268509
:103660001925230A2401E5B7EFC2FFCE2A84EFF023
:103670005FFB9145130544007D286FC01FD09C411E
:10368000938787FB138787046314B7002E8739A0BD
:103690000346150283C617026371D602F447130668
:1036A0008504F0C738C574C590C2834705026CCD48
:1036B00093E727002300F5028280BC47D1B71C4165
:1036C0006309F500138787FB294509C703C597FDE3
:1036D0008280294582807C4538455CC398C38347F6
:1036E0000502232E0504F59B2300F5028280EFC21C
:1036F0009FC6784534456C4DD8C214C3EFF03FF8EF
:103700006FC0BFC7EFC23FC5834705022A84898BBC
:1037100081C72CD1EFF03FFC83470402858B81C722
:103720002285EF00A07283470402918B99E32285E2
:1037300015226FC09FC4EFC21FC21C41AA842E89EC
:103740008043138587FB130484FB930785046394EC
:10375000F4006FC09FC2CA85EFF0DFFA3C442285B7
:10376000138487FBDDB793575500D10737670020D7
:10377000130787B18A07BA971346F5FF8546B396B4
:10378000C6009043D18E94C3834747056374F50008
:10379000230AA7048280B7670020138787B1834775
:1037A00047058E07BA978843130585FB82803767E4
:1037B0000020930787B1A946238AD704130787B14E
:1037C000938607059CC3DCC3A107E39DF6FE23286F
:1037D00007048280EFC29FB62A8903451502B767A6
:1037E0000020938487B193193500CE9498401384B8
:1037F00087B16394E400EFF01FF7B30734019443FB
:1038000013078904D8C22324D9042326990498C312
:103810006FC01FB6EFC29FB22A8903451502B76772
:103820000020938487B193193500CE949840138477
:1038300087B16394E400EFF01FF3B3073401D8437A
:1038400093068904D4C3232499042326E90414C3CA
:103850006FC01FB2EFC23FB083A741850347150277
:1038600083C717026316F700EFF0DFFA6FC0FFB0EF
:10387000EFF05FF6E5BFEFC21FAE2A84952A25E977
:103880007C44384403461402B76400205CC398C3E8
:10389000138784B193173600BA979843938484B101
:1038A0006311F70293575600D1078A07A6978546FA
:1038B0001347F6FF3397E60094431347F7FF758FDE
:1038C00098C383C744056394C702B76700200144C7
:1038D000938787B631A0130404021374F40F910781
:1038E000884375D9EF00700B2295238AA4046FC01A
:1038F000DFA801A003A7C1858547631BF70083C725
:1039000081859306900F63E5F6008507238CF1848B
:10391000828003A7C18585476314F704EFC2BFA364
:10392000EF00807983C781852A8489E7EF00807959
:103930006FC0BFA4FD1793F7F70F238CF184FDF739
:1039400083C74186E5F7EFF01FE523A0A18683A793
:1039500041856314F5002285D1BFEF002078E5BFD3
:103960008280EFC25F9F83A7C18585441305501FE6
:10397000638D9700EFF03FE223A0A18623AAA184E4
:1039800023AE9184EF00407601456FC01F9F03A5D1
:10399000C1857D1513351500828003A7C185854734
:1039A000631DF70283C7818503C74186D98F95E7D9
:1039B000EFC27F9AEF0040702A84EFF0DFDD23A092
:1039C000A18683A741856317F5002285EF00806FEC
:1039D0006FC0BF9AEF00C06FCDBF828003C5418624
:1039E0003335A000828003C581853335A0008280F5
:1039F000B77700209387879F1D8D13351500828030
:103A000083A741853385A740133515008280EFC217
:103A10009F9403A8418483A7018437460000B7C55B
:103A20000000377500208148254781461306268F00
:103A3000938585501305859F2D206FC01F94EFC27D
:103A40009F91EF00606CEFF09FD6377500208D6579
:103A5000130505A7EFF03FBB19E1EFF05FFB6FC067
:103A6000DF91EFC2BF8D2A842E8B3289B68ABA8449
:103A7000BE89428AEFF03FF769E91305C0445DC88B
:103A8000630A090A6388090A9307F0071305407758
:103A900063F2470BA5476391F40A2285EFF05FF5C7
:103AA00051CD930704043CC07CC0930784043CC4FC
:103AB0007CC4930704053CC87CC8A947230CF404C4
:103AC00083A601811307C40223200406232E0404C5
:103AD0002322040623240406D8C254D43746000007
:103AE0009386018123A8E18014D85287CE861306DD
:103AF000E6C2D6854A85EF00A0643D46DA8508C057
:103B0000A3009402232C2401232E540123223403E6
:103B10002324440313058400EF40E015712BAA848D
:103B2000230004022285EFF0FFCE2685612BEFF003
:103B30001FE601E96FC0DF83E3F597F61305F07622
:103B4000D5BFEFF09FE50145F5B713050019DDB7C7
:103B5000EFC2CFFE2A84EFF01FE99307001911EDA1
:103B600019E003A441852285EFF09FE911E9228540
:103B7000EFF01FE89307D07611C93E856FC04FFF65
:103B8000EFF0DFE59307406A7DD1C5BF35233C48A0
:103B900013090405AA89631DF9068347040281E716
:103BA0002285EFF05FCD83470402858B99C3228580
:103BB000712C83470402898B81C72285EFF0BFB146
:103BC0001C5858544E855CC398C39307C4025CD4F8
:103BD0001CD8930704043CC07CC0930784043CC4F5
:103BE0007CC4A947230CF404A1472300F402232832
:103BF0002405232A240523200406232E040423223B
:103C00000406232404067D29EFF03FD98147B5B788
:103C10008443138587FEA11493078501E30FF9F60A
:103C2000EFF09FA49C4C2685938487FEF5B7EFC2E6
:103C30008FF20145EFF0DFF16FC02FF4EFC2AFF16B
:103C4000EFF07FDA19ED8D29AA8403A54185EFF005
:103C50009FC203A54185EFF0FFBB2685A521EFF0AC
:103C6000DFD36FC08FF1EFC26FED2A84AE89EFF022
:103C70009FD75DE51305C04405C0A1471305F07645
:103C800063EC3701152983471402AA8A6398370128
:103C90001529EFF09FD001456FC08FED2448130A1E
:103CA0000405631F9A004E898347040213F7270017
:103CB00021C3A30024032285EFF07FA35685C9BF4B
:103CC000A1142949938784016317FA00E37D39FD24
:103CD000230C3405D1BF13854400EFF05F9EAA8703
:103CE0006373A900CA87844C13F9F70FA114D9BFD5
:103CF00013F7170001C7A3002403C9B7E1F3228516
:103D0000EFF07FB72285A3002403EFF07FCF09C532
:103D10002285EFF03FAC5DB72285EFF0BFAF79BFF2
:103D20001305001995BFEFC26FE12A84AE84EFF04E
:103D30009FCB9307001901EDEFF05FCA9307406A2C
:103D400019E5B367940099E7EFF05FEF81473E858F
:103D50006FC00FE2FD576316F40093075006E38827
:103D600084FE992EAA8903A54185A285268611285D
:103D700003A54185EFF03FB04E85A926EFF0FFC1C6
:103D8000F1B7EFC24FDD41112A842EC632C42D2671
:103D900083A78181B2452246938707FC0CDC50DC67
:103DA0008146014713838181138E070463116E06D8
:103DB000B388D540B3BE15013308E6403308D84177
:103DC000232C1403232E040363016E02B385B64033
:103DD000B3B6B600118F158F945FD05FB695B3B6AA
:103DE000D500329736978CDFD8DFF843930604046A
:103DF000F4C32320C40578C014C3E9248347040214
:103E000093E717002300F40241016FC00FD783A886
:103E1000870383AEC703B69833B8D800BA9E7698A6
:103E2000E36806F96314C800E3E415F9639A150121
:103E300063180601034F140283CE1702E36ADFF70B
:103E4000BC43C6864287938707FCB9BFEFC2AFD099
:103E50002A849D243C40130704046388E7041387E5
:103E600007FC21C7138781816381E704145C8328E1
:103E7000C403F9553383D54003A6C7FF33B86500A3
:103E800093C5F8FFB385054103A787FF63EAC50221
:103E90006314B6006366E302BA9633B7E60046964B
:103EA000329723ACD7FE23AEE7FE7840D8C31CC3BD
:103EB000112C83470402F99B2300F4026FC0EFCB5F
:103EC0007956FD5623ACC7FE23AED7FEF9BFEFC22D
:103ED0008FC841112A842EC6C52283A7818683A656
:103EE000C186B24533868700B337F600AE96B697E3
:103EF00023A6F18683A7818123A4C186938481812F
:103F000063969700C12241016FC02FC703A7C7FF67
:103F10002A8983A687FF138507FC63EFE5026314F4
:103F2000B700636BD40280438146014723ACD7FEC0
:103F300023AEE7FE130404FC93070504638897028D
:103F40001C5D585DD98F9DE38945EFF0AFFB3C4088
:103F50002285138407FCCDB733848640B3B6860030
:103F60000D8F158F23AC87FE23AEE7FE4A8559BF20
:103F7000EFC26FBEEFF0BFA109C505458145EFF067
:103F80001FF56FC08FBF21651305058073150530C0
:103F9000828073100530828037F700E01C4386076B
:103FA00085831CC3828037F700E01C43B70600807E
:103FB000D58F1CC38280EFC20FBAEFF0DFFE6FC057
:103FC000CFBBB7F700E023A0070023A2070081467C
:103FD00094C70147D8C71306F5FF90CB8146D4CBD1
:103FE0003D4798C382801375F50FB7E700E023863D
:103FF000A7408280B7E700E041572387E740056785
:1040000023A0E710116723A0E7108280197182FEB8
:1040100086FC8AFA8EF892F696F49AF29EF0A2EE58
:10402000A6ECAAEAAEE8B2E6B6E4BAE2BEE042FE28
:1040300046FC4AFA4EF852F656F45AF25EF062EE38
:1040400066EC6AEA6EE872E676E47AE27EE08A82FC
:1040500003A1018216C0EFF09F9319C9EFF09F8969
:10406000B7F700E023A20700EFF09FF0EFF07F8AA0
:1040700002417670E6705671C6713672A67216737A
:1040800086737664E6645665C6653666A666166708
:1040900086677278E2785279C279327AA27A127B94
:1040A000827B726CE26C526DC26D326EA26E126FC8
:1040B000826F096173002030EFC2EFA9EFF0BFEC0F
:1040C0006FC0AFABEFC22FA9EFF0BFEC6FC0EFAA8C
:1040D000EFC26FA8EFF03FED6FC02FAAEFC2AFA7FE
:1040E000EFF07FED6FC06FA9EFC2EFA6EFC04F9169
:1040F000EFC26FA62A841305000FEFF0DFEE2285D2
:10410000EFF03FEC6FC06FA7EFC2EFA413870182FF
:104110001C438145F117F19B1CC3B707002003A680
:10412000871E83A6C180B707002003A5071E492369
:1041300023A8A184EFF0DFFBEFF0DFEB6FC0EFA36C
:104140003697719BB7E8EAAC2A8E130847F8130537
:1041500007F885462943938808D0930E0002B3C719
:104160006602110833EF660292078506B3E7E7019E
:10417000B3E71701232EF8FEE393D6FF8E8723269D
:10418000F7F8A167938707882324B7FA2324C7F891
:104190002322F7F82320C7F982804177698FAA8705
:1041A000014519E3C2074145370700FF7D8F19E339
:1041B000A2072105370700F07D8F19E3920711054B
:1041C000370700C07D8F19E38A07090563C607001A
:1041D00099C3050582800905828001A001A001A084
:1041E00001A001A001A001A001A001A001A001A0C7
:1041F00001A001A001A001A001A001A001A001A0B7
:1042000001A001A001A001A001A001A001A001A0A6
:1042100001A001A001A001A001A001A001A001A096
:1042200001A001A001A001A001A001A001A001A086
:1042300001A001A001A001A001A001A001A001A076
:1042400001A001A001A001A001A001A001A001A066
:1042500001A001A001A001A001A001A001A001A056
:1042600001A001A001A001A001A001A001A001A046
:1042700001A001A001A001A001A001A001A001A036
:1042800001A001A001A001A001A001A001A001A026
:1042900001A001A001A001A097C1FF1F938181741B
:1042A00017C10020130101D6178500001305057FF3
:1042B00097C5FF1F938505D51386018563FAC50051
:1042C0008322050023A0550011059105E3EAC5FEF0
:1042D00013850185976500209385059A6377B5005E
:1042E000232005001105E36DB5FEFD42739002BC6D
:1042F000FD4273904280B78200009382028073A0D7
:10430000023097C2FFFF938262D393E23200739030
:104310005230EFC08FAA97C2FFFF9382821F739023
:104320001234730020309C4513F7070113F8F7008F
:1043300001C7D8413368E8008E2113F7F50F39C360
:1043400018418146854E3D4F930F800293028004B1
:10435000214E3396DE00B3F8C5006311160393981F
:10436000260033131F011343F3FF3377E300B31821
:10437000180133E7E800639FF70550C98506E39A03
:10438000C6FD18C11307F00F6375B70454412146E9
:10439000854E3D4F930F800293028004414EB398A7
:1043A000CE0033F715016392E802131726000117B8
:1043B0003313EF001343F3FFB376D3003317E80052
:1043C000D98E639DF701232A15010506E319C6FD61
:1043D00054C18280E39457FA10C94DB7E39757FE52
:1043E00023281501DDB7371702405C439146B18B96
:1043F0006385D700A1466382D706B7177A009387F3
:1044000007201CC1371602405C4237070020130703
:1044100007009183BD8BBA9794231C41B3D7D70073
:104420005CC15442A1829D8ABA969422B3D6D70029
:1044300014C55442AD829D8A36971823B3D7E7003E
:104440005CC558423983937637001387418236978B
:104450001823B3D7E7021CC982805C4354434167E9
:10446000C983F98E37F7FF1F0327C770BD8B8907F4
:104470001316170163480600454601476392C702B9
:10448000C94739A809476389E7023D476388E702BE
:1044900041476388E702454601476393C700C14728
:1044A00085E6B746024083A60680C18A8DC6B71648
:1044B0007A009386062025A00147D9B70547B5475E
:1044C000C5B70147BD47E9BFB7160240D4421396AE
:1044D000E600E35E06FCB7163D0093860690B387C0
:1044E000D7021CC105D31C41858321BF99C537174D
:1044F00002401C4F5D8D08CF8280B7170240984F55
:104500001345F5FF798D88CF8280EFB2DFE416295D
:10451000F577FD17F58FF621DA257971D58F1EA96C
:104520005625FD779387379FF58FD6212A842EC68F
:10453000D58F9625D58FB625D58F5EA55E29C20766
:10454000C18393F7F7CFD98F5EA96808EFF0BFE971
:10455000B747014093870780B245631AF404A25716
:1045600056246547B387E702C206C186984163D2E5
:104570000604060752244206B3D7E7021307400693
:104580004186B3D6E702B3F7E70292066355060207
:104590008E0793872703B3D7E70213F77700B36734
:1045A000D700C207C1831EA445616FB01FDD9257BB
:1045B00045BF0A07C1B7920793872703B3D7E7021E
:1045C000BD8BD58FF9BF91C55E250967D98F5EA5D3
:1045D00082805A25F977FD17F98FD5BF93F5F51F1E
:1045E0004EA182800A216D8D3335A0008280EFB20A
:1045F0009FD62A841165011185451105EFF01FEF43
:10460000930700207C82371501408D473EC44C0043
:10461000E147130505803EC6EFF0FFD022C83744BE
:104620000140B70708000C08130504803ECC02CAFD
:10463000231E0100EFF07FED854513050480EFF0A8
:104640009FF805616FB07FD3EFB25FCFB7440140F1
:10465000AE893289014493840480634524014A85EC
:104660006FB01FD1930500042685EFF0BFF77DD909
:10467000B38789008385070026850504C205C181AB
:10468000EFF0DFF5D9BF138781821C43B7A6002066
:10469000938646C73E95636BD500B7B600209386D8
:1046A000060063E5A60008C33E858280FD57EDBF86
:1046B000B687B2882A832E88639D061463F9C50ADB
:1046C0004167636EE61AB70700016363F6349356D9
:1046D0008601E147178700001307C7EB36970347AA
:1046E0000700BA97130700021D8F19CB3398E50016
:1046F000B357F500B318E60033E807013313E500BC
:1047000013D608013355C80293960801C182935706
:1047100003013377C802B385A60242073368F70066
:10472000637AB80046989307F5FF636418016367DE
:10473000B8303E853308B8403357C802420313539C
:1047400003013378C802B386E60242083368680082
:10475000637BD80046989307F7FF636518017917C4
:104760006363D8003E874205598D8145828001E60A
:104770000547B358C702416763EAE80EB70700016F
:1047800063ECF82893D68801E147178700001307E8
:1047900067E0369783460700BE9693070002958F21
:1047A000E5EB939E08013387154113DF080193DE83
:1047B0000E018545935703013355E7033377E7032C
:1047C000B306D5034207D98F63FAD700C6971307FC
:1047D000F5FF63E4170163E6D7263A85958F33D753
:1047E000E703420313530301B3F7E703B30ED70301
:1047F000C207B3E7670063FBD701C6979306F7FFCD
:1048000063E51701791763E3D70136874205598DB0
:10481000828063E2D504C16763E2F604B707000152
:1048200063E4F61E13D786016148978700009387DB
:1048300067D6BA9703C70700130E00024297330EDC
:10484000EE40631A0E0C63EDB61C3335C5001345FC
:104850001500814582808145014582809307F00FD4
:1048600063F3D71C13D786002148C1B71307F00F95
:10487000C686E37C17F193D68800A14739B71307A2
:10488000F00FB286E378C7E493568600A14799B546
:10489000B398F80033D6D50013DF0801335EE60382
:1048A0003397F500B356D500558F939E080193DEDC
:1048B0000E013313F50093550701B376E603B38772
:1048C000CE03C206CD8E63FBF600C6961306FEFF2E
:1048D00063E4161763F2F616791EC6969D8E33D6DC
:1048E000E60393170701C183B3F6E6033385CE02CF
:1048F000139706015D8F637BA70046979307F6FF2A
:10490000636817136376A7127916469793150E01FD
:10491000098FD18D45B5B357E600B396C601DD8E3C
:1049200033D3E50013DF0601B357E303939E06017B
:1049300093DE0E013398C5013357E5003368070154
:10494000935808013316C6013373E303B385FE029F
:104950004203B368130163FBB800B6981387F7FFEF
:1049600063EAD80C63F8B80CF917B698B388B84066
:1049700033D7E803420813580801B3F8E803338338
:10498000EE02C208B3E5080163FB6500B6951308A3
:10499000F7FF63EDD50863FB65087917B695C20785
:1049A000416FD98F1307FFFFB3F6E70093D80701D4
:1049B000718F4182B38EE602B3856540B386C6022D
:1049C00013D80E013387E802BA96C2963386C8021E
:1049D00063F3E6007A9693D80601469663E2C50231
:1049E0006385C5003E858145828041677D17F98ECC
:1049F000C206B3FEEE003315C501F696E374D5FE8C
:104A00001385F7FF8145828013D70601414831BDE8
:104A100093560601C1477DB993D60801C147B5B386
:104A20008145054582803687014801B5428785BFAB
:104A30003E86E9BDBA871DBF328E4DB579154698C1
:104A4000D5B97915C69759BB3708100001117D18E3
:104A50003377B80026CA3378D80093D4450113D3EE
:104A60004601131E37004EC61357D5010E08935743
:104A7000D60193F4F47F1373F37F06CE22CC4AC899
:104A800093D9F50193DEF6013367C701131F350093
:104A900033E80701931F3600338E64406380D919D1
:104AA0006356C0136304031CB70680009307F07FAE
:104AB0003368D800638FF4369307800363C0C7352B
:104AC000FD4763CDC747130500023305C541B3D782
:104AD000CF01B316A8003399AF00DD8E3339200122
:104AE000B357C80133E926011D8F33092F41B3376E
:104AF0002F013306F7409317860063D40724370746
:104B000080007D173374E600630C042C2285EF10BF
:104B1000D031130785FF93070002998FB357F9002F
:104B20003316E400D18F3319E9006341972A330526
:104B30009740130615007D47634DC73813070002E1
:104B4000118FB356C9003319E9003397E700558F29
:104B5000333920013369270133D6C7008144937765
:104B6000790081CF1377F90091476308F7001307A5
:104B70004900333927014A963A899317860063D64C
:104B8000071C138514009307F07FCE856304F5207E
:104B9000B70780FFFD17F18F9398D701135939009C
:104BA000A607B3E82801B1831375F57F9396C70074
:104BB0005205F2406244B182FE05C98ECD8ED244C8
:104BC0004249B2494685B68505618280631E0E0A58
:104BD000138314001373E37F63170322B367E701A2
:104BE000B368F801639D041A63870740638608442D
:104BF0003309FF41B307074133362F013386C740DE
:104C00009317860063D6074C3389EF41B307E8401A
:104C100033B62F013386C740F68991B76350C00F72
:104C20006300030CB70680009307F07F3368D80059
:104C3000638AF43A9307800363CBC713FD4763DFAE
:104C4000C73513090EFE93070002B3562801630A05
:104C5000FE00130900043309C94133192801B3EFD9
:104C60002F013339F0013369D90031A2B367F8015C
:104C7000638A071C9307FEFF638C07389306F07F57
:104C80006309DE1A3E8E0DBDB30593406391042285
:104C9000B367E701638707329387F5FF63810744B2
:104CA0009306F07F638CD520BE859307800363CC89
:104CB000B72AFD4763CFB73C930700028D8F3319A6
:104CC000F700B356BF00B317FF003369D900B337FD
:104CD000F0003357B7003369F9003308E84041ACBE
:104CE000B367F801638007349307FEFF638A0720E8
:104CF0009306F07F6308DE2E3E8E2DBF631E0E14DA
:104D00009386140093F7E67F63910734B367E70156
:104D10006395042C6380073EB367F801638E073008
:104D20003309FF01B3070701333FE9013386E70188
:104D30009317860063D70700B70780FFFD177D8EA6
:104D4000854493777900E39F07E09317D601935842
:104D50003900B3E8F800935736001307F07F638DEE
:104D6000E404B207B18313F5F47FCE8581B53369CE
:104D7000F801333920017A99B337E9013386E70026
:104D800093178600E3DF07FA85049307F07F6396A5
:104D9000F418CE851305F07F8147814801BDC1EB32
:104DA0006384083A931636009317D8018D82B3E8CE
:104DB000D700F68993573800B3E7F800F9DB81454F
:104DC0001305F07FB70708008148CDB3370680FF91
:104DD0007D167D8E93777900998CE39507D8B5B7CA
:104DE0004A85EF10900413078501FD47E3D5E7D20C
:104DF000130685FFB317C900014905BB3369F801E4
:104E000033392001DDB13309FF4133060741333423
:104E10002F01330486409317840063CD0724B368C1
:104E20008900E39308CE8147814981441DBFE398FF
:104E300008F80E059317D7010D81B3E8A700935723
:104E400037009DBF0E059317D7010D81B3E8A7006A
:104E5000F2849357370011B73305934063820412ED
:104E6000B70680009307F07F558F630DF32E9307ED
:104E7000800363CBA720FD4763C3A72A93070002E3
:104E8000898F3319F700B356AF00B317FF003369AA
:104E9000D900B337F0003357A7003369F9003A98C7
:104EA0007E99B337F901338607019A84D1BDB706DD
:104EB00080009307F07F558FE319F3DE93173600D8
:104EC0008D839318D801B3E81701F68993573800FA
:104ED000E5B5130715FE9306000233D7E700630A12
:104EE000D600930600043386C6403396C700336964
:104EF000C900333920013369E9000146814491B585
:104F00003309FF01B30707013336E9013E969317D2
:104F100086008544E3D707E28944B70780FFFD1781
:104F2000F18F1357190013791900336927019398EA
:104F3000F70133E9280113D6170015B113090EFE46
:104F400093070002B3562801630AFE001309000408
:104F50003309C94133192801B3EF2F013339F00167
:104F60003369D90059B63369E701333920013389F0
:104F70002F41B3B72F013306F8409A84F689A5BEB6
:104F8000B367E701638207189307F5FF6384071C83
:104F90009306F07F6304D5123E85D1BD93070002CE
:104FA000B387C741B316F8003399FF0033D6CF015A
:104FB000D18E33392001B357C80133E926013E971A
:104FC0005DBB931736008D839318D801B3E81701A2
:104FD000AE8493573800F68949B3EDC33369F801BD
:104FE000E31F09DC0E059317D7010D81B368F500A7
:104FF00093573700D1B36381080E93163600931789
:10500000D8018D82B3E8D700F6899357380091BB59
:105010003309FF41B3070741333F2F013386E7418F
:105020008544D1BC0E059317D7010D81B368F500F7
:10503000F2849357370015B30E059317D7010D81EE
:10504000B3E8A7009357370029BB9307F07FE382AB
:10505000F6D43309FF013336E901B3070701B297EC
:105060009398F7011359190033E9280113D6170053
:10507000B684C1B93389EF413307E84033B62F0115
:105080003304C740F68949B43369E7013339200155
:1050900001BD938705FE93060002B357F700638AAC
:1050A000D50093060004B385B6403317B700336FBD
:1050B000EF003339E0013369F90055BD931736002D
:1050C0008D839318D801B3E8170193573800EDB1D9
:1050D000B368C900E39708C68147814959B133894C
:1050E000EF41B307E84033B62F013386C740F68956
:1050F000854411B4931636009317D8018D82B3E816
:10510000D70093573800B1B9931636009317D801DA
:105110008D82B3E8D700AA84935738003DB993072E
:1051200005FE93060002B357F700630AD500930605
:1051300000043385A6403317A700336FEF003339DF
:10514000E0013369F900A9BB81451305F07FB7077A
:105150000800A9BC3309FF01B30707013336F90181
:105160003E9675B3931636009317D8018D82B3E837
:10517000D7009357380089B1397193D7450122DCA4
:105180004AD856D22A891394C50006DE26DA4ED6AE
:1051900052D45AD05ECE13F5F77F318093DAF50101
:1051A000630B05109307F07F630BF514135AD901B5
:1051B0000E0433648A00370A8000336A4401131BEB
:1051C0003900930415C00144814B13D8460113994B
:1051D000C6001378F87FB2881359C90093D9F60135
:1051E000630E08089307F07F6300F8041357D60195
:1051F0000E0933692701130818C0B7078000336709
:10520000F90093183600B38404418145BD4733C883
:105210003A0163E4871A977700009387A72F0A045F
:105220003E9410403E9602863367C90093841480F2
:10523000631207101364240081488945C1BF130617
:10524000F07F81470147B207F25062545206B183A2
:105250007E08D18FB3E70701D2544259B259225A7E
:10526000925A025BF24B3A85BE85216182800148E9
:105270001306F07FB70708000147F1B73367C9008D
:105280004DC7630809304A8532C4EF10003A224600
:10529000130755FFF547930685FF998F3319D900FA
:1052A000B357F60033E72701B318D60026959304C9
:1052B000353F8145A1BF336A240163030A0636C620
:1052C00032C46306042A2285EF1020362246B246F5
:1052D000AA84130755FF754A138B84FF330AEA40EB
:1052E00033146401335A4901336A8A00331B69015C
:1052F0001305D0C0B30495400144814BF9B5336A1E
:10530000240163180A002144014B9304F07F894B68
:105310006DBD228A4A8B31449304F07F8D4B75B565
:105320001144014B8144854B4DB5136414008148F1
:105330008545E9BD136434004A878D45C1BD630AC4
:10534000052E8547898F9306800363DDF63201467B
:1053500081470147CDBDCE868947638DF53A8D479C
:10536000E387F5F085473688E383F5FE1385F43F40
:10537000E357A0FC93F778006396072893D638008C
:105380009317770063D80700B70700FFFD177D8FDD
:10539000138504409307E07FE3C3A7EA1316D70100
:1053A00093179700B1833367D6001376F57F61BDFD
:1053B000D6865287DA88DE8545B763614723630D59
:1053C000EA20DA86FD145284014B9317870013D329
:1053D00088013363F300935E0301B357D403131FB3
:1053E0000301135F0F0193D50601139E88003374E8
:1053F000D4033307FF024204C18D63FBE5009A9595
:105400001386F7FF63EE652663FCE526F9179A9588
:10541000998D33D7D503C206C182B3F5D5033306C0
:10542000EF02C205D58D63FBC5009A959306F7FF81
:1054300063E6652463F4C52479179A95C20741642D
:105440005D8F9307F4FF3375F70093580701935F5F
:105450000E01B377FE00B302F502B386C540B383F5
:10546000F80293D502013386AF021E962E9633853D
:10547000F803637376002295C168FD189355060101
:10548000337616014206B3F81201AA95469663E6F2
:10549000B6126382B6123306CB408D8E333BCB00FF
:1054A000338B66411385F43F630C6317B358DB03FA
:1054B00093550601337BDB03B3061F03420B33EB2B
:1054C0006501637BDB001A9B9385F8FF636D6B209E
:1054D000637BDB20F9181A9B330BDB40B356DB03ED
:1054E00042064182337BDB03330FDF02420B33661C
:1054F0006601637BE6011A969385F6FF6367661E75
:105500006375E61FF9161A96C208B3E8D80093959A
:10551000080193D20801C181B38EF5023306E6413A
:10552000B385BF0293D60E01B387F202BE95AE9645
:10553000B38F5F0263F4F600C167BE9FC165FD15BE
:1055400093D70601ED8EC206B3FEBE00BE9FF6964F
:10555000637FF6091A969387F8FF6369661A636892
:10556000F619630FF61BBE8893E8180011B54A853B
:10557000EF10A00B13075501F145930405022246D5
:10558000B246E3DAE5D4130485FF331A8900014BF0
:1055900085B3328532C4EF10400913075501F14637
:1055A000AA87224613050502E3D6E6CEE117331794
:1055B000F6008148E5B9E370CBEE729B3335CB0141
:1055C0001A95AA961305F7FF6378D30263E6B6101F
:1055D0006382D5102A87C1B5E3651BDF93551B0095
:1055E0009316FA0113541A00CD8E7E0BF9BBE31DFE
:1055F000F6F7E38F06D6B9BFE31ED3FCE378CBFD05
:105600002A8751BD93F7F8009146E389D7D693B71F
:10561000C8FF9386480093C717008D823E978DB3CD
:1056200081468547E34CA0FEFD58E31C05D093045A
:1056300010C085471385E441B316A70033D6F800A0
:105640003395A800D18E3335A000C98E13F67600AD
:105650003357F70001CE93F7F60011466388C70071
:1056600093874600B3B6D7003697BE869317870058
:1056700063D80704054681470147F1B636877DBBED
:10568000B28779B3FD46E3D7F6FA0556098E93063D
:1056900000023356C7006388D7009387E443B317EB
:1056A000F700B3E8F800B3361001D18E13F6760098
:1056B000814701CE93F7F60011460147E392C7FAFE
:1056C000931797001316D701B18313D73600518F64
:1056D000014695BEE370CBF0729B3335CB011A9532
:1056E0007917AA964DBBAE88C5BBAE8631BD931760
:1056F0001E0033BEC70172931A96F9183E8EE31549
:10570000F6E7E307DEC693E818009DB1BE88E30A1A
:10571000F6FF99BD36881306F07F8147014725B60D
:10572000E367DEFCBE88E310DEFE99B113D74501C6
:10573000B7071000FD1713D846011377F77F9308BA
:10574000F07F33FEB700AA8EF58FFD81328F13787C
:10575000F87FFD82630B170105436306180163148C
:105760000701630DFE001A858280B368AE00054311
:10577000E39B08FEE319E8FED18FF5F70543E394B8
:10578000EEFF0143E381D5FE054371FF3365AE00B3
:105790003333A000C9BF13D74501B7071000FD1769
:1057A00013D846011377F77F9308F07F33F3B700E0
:1057B0002A8EF58FFD81B28E1378F87FFD82630803
:1057C0001703630018030DEBB368A300631408000C
:1057D0005D8E29CA638508046388D502054595ED69
:1057E0008280B3E8C700E38008FE79558280336584
:1057F000A30065FD630CE802631408005D8E79DE8A
:10580000E39ED5FCE34CE8FC63480701E3E867FC52
:105810006303F302637FF30081E57D558280F5DE4B
:10582000054582800145E39B08FA82805D8E69DA36
:105830006DBF01458280E3E3CEFB0145E372DEFBF1
:10584000E5F1E1BF13D74501B7071000FD1713D8E5
:1058500046011377F77F9308F07F33FEB700AA8ED7
:10586000F58FFD81328F1378F87FFD82630E170369
:10587000630D180129E3B368AE00631F08005D8E55
:1058800001EE0143638C080421A8B3E8C700094373
:10589000639608046DD305A0638408046385D5026C
:1058A00005438DCD7D531DA8B368AE0009436397B2
:1058B0000802630AE802631408005D8E75D2E39162
:1058C000D5FEE34FE8FC63490701E3EBC7FD630F37
:1058D000FE0001436374FE00F1D505431A85828002
:1058E000EDFE7D53E5BF5D8E79DACDBFE36ADFFB68
:1058F0000143E3F5EEFFF5F175B739714AD813D9D5
:1059000045014ED652D456D29399C50006DE22DC0C
:1059100026DA5AD05ECE1379F97F2A8A93D9C90044
:1059200093DAF501630D090E9307F07F6306F9180A
:105930001354D5018E09B36934013704800033E470
:10594000890093143500130919C08149814B13D77D
:105950004601139AC6001377F77FB285135ACA001F
:1059600013DBF601630B07109307F07F6303F70463
:105970009357D6010E0A33EA4701130717C0B7073A
:105980008000B367FA00931536003A99814833C70F
:105990006A01BD463A851308190063E83617177681
:1059A0000000130626BB8A09B29983A60900B296A5
:1059B0008286B367CA001309F97F6399071293E9D6
:1059C000290081458948E1B701479307F07F3704F3
:1059D000080081443204D20731807E075D8C598CE7
:1059E000A285F250625426854259D254B259225AA5
:1059F000925A025BF24B216182805A853E84AE84CA
:105A0000C68B8947638DFB0E8D47E38FFBFA854775
:105A10002A87639EFB3881470144814465BF33E494
:105A2000A90061C036C632C4638C092A4E85EF00D6
:105A3000D03F2246B246AA87130755FF7544938488
:105A400087FF198CB399990033548A003364340169
:105A5000B3149A0013D746011309D0C0139AC60095
:105A60001377F77F3309F9408149814BB285135A87
:105A7000CA0013DBF601E31907EEB367CA00B1C72A
:105A8000630F0A22528532C4EF00303A22462A8739
:105A9000930655FFF547930587FF958F331ABA0094
:105AA000B357F600B3E74701B315B6003309E94031
:105AB0001309D9C08148E1BD33E4A90001ECA14933
:105AC00081441309F07F894B59B593E91900814549
:105AD000854875BD4E84AA84B1491309F07F8D4B6A
:105AE000BDB5914981440149854B95B593E939008C
:105AF000D2878D4869BD89475685E397FBF02A8791
:105B00009307F07F01448144F1B5C16E1386FEFF17
:105B100093D6040113DE0501F18CF18D33869502D5
:105B20003383B6029358060133059E021A95AA984C
:105B3000B382C60363F36800F692C16F1383FFFF5D
:105B400033F5670093D30701B3F76800C2073373D7
:105B500066003E933306950293D80801B387A602E8
:105B6000135F0601B3849302BE94FA94B38E760257
:105B700063F3F400FE9E416A9307FAFF935F04010A
:105B8000B376F400B3F9F4007D8EC1803384D5027E
:105B9000C209338FD401B299CE98B307DE02935E67
:105BA0000401B385BF02AE97BE9E330EFE0363F3BE
:105BB000BE00529EC1679385F7FF33F6BE006D8C21
:105BC0004206229693DE0E01B305D502769E3385FA
:105BD000AF0213D40501B386D302AA96A296B38F5F
:105BE000F30363F3A600BE9F41657D15B3F7A600DE
:105BF000C2076D8DAA97B3855800B3B93501FA97DE
:105C0000B2953384370133B6C500B30EC401338572
:105C1000CE0033343401B3B7E701C18F33BECE01B8
:105C200013D406013336C5003E943366CE009394F8
:105C3000950032947E94B3E4640026049356750173
:105C4000B3349000DD8193179500CD8C558CDD8C9D
:105C50009317740063DB070093D7140085889316AD
:105C6000F401DD8CD58C058042899307F93F635997
:105C7000F00893F6740081CE93F6F4001146638821
:105C8000C60093864400B3B496002694B684931657
:105C9000740063D80600B70700FFFD177D8C9307DB
:105CA00009409306E07F63CFF60E93D63400931439
:105CB000D4012604D58C318093F7F77F21BB328540
:105CC00032C4EF00901693065501F1471307050201
:105CD0002246E3D1D7DC6115B317A6008145F9B39D
:105CE000EF00B01413075501F14593070502224652
:105CF000B246E3D5E5D461153314AA00814499BBBB
:105D000085469D8EB1E71309E941B3972401B3D4C9
:105D1000D40033192401B337F000B3649900DD8C4B
:105D200093F77400B356D40081CF93F7F400114673
:105D30006388C70093874400B3B49700A696BE84D7
:105D40009397860063D8070485470144814459B17D
:105D500013068003E341D6CC7D46E356D6FA0556BA
:105D6000B307F640930500023356F4006387B6008C
:105D70001309E943B3172401DD8CB3349000D18CAF
:105D800093F67400014499CA93F7F40011468146D2
:105D9000E392C7FA139496003180F6068D80D58C75
:105DA00081470DB99307F07F0144814425B14289B1
:105DB0006DBD370710007D1701113373B70093D8FD
:105DC0004601758F935ED60122CC26CA0E0393D46A
:105DD00045019357D5010E0706CE4AC84EC693F823
:105DE000F87F130EF07F33E7EE0093F4F47F13D4C3
:105DF000F50133E36700131F3500FD82931E360063
:105E0000638FC81793C61600B38514416304D41278
:105E10006350B018638A081AB70780005D8F638FDC
:105E2000C4579307800363C2B734FD4763C3B748C1
:105E3000930700028D8FB3D9BE003318F700B39ECD
:105E4000FE00336838013357B700B339D0013368E7
:105E500038013303E340B3090F41B3373F01330641
:105E6000F3409317860063D20724370980007D1919
:105E700033792601630E092C4A85452F130785FFC8
:105E800093070002998FB3D7F9003316E900D18F39
:105E9000B399E9006344972A058F13061700FD465E
:105EA00063C4C63A13070002118FB3D6C9003398F2
:105EB000E9003397E700558F33380001B3690701D4
:105EC00033D6C700814493F7790081CF93F6F90068
:105ED00091476388F6009386490033B836014296AD
:105EE000B6899317860063D6071C1387140093079F
:105EF000F07F05886306F720B70780FFFD17F18F55
:105F00001398D70193D93900A60733683801B183B4
:105F10001377F77F9396C7005207B1827E04D98E1C
:105F2000C18EF2406244D2444249B2494285B685AC
:105F3000056182806356B00A638A0812B707800041
:105F40005D8F6386C42D9307800363C7B718FD4731
:105F500063D1B73C138805FE93070002B3590701CC
:105F6000638AF50093070004B385B7403317B70081
:105F7000B3EEEE003338D0013368380195A2B36731
:105F8000D7019385148099E393C61600630AD4045D
:105F9000D1E19387140093F7E77F6398071EB367F7
:105FA000E3013368D701639204166381073C6315EC
:105FB0000842131835009316D3011358380033E8FC
:105FC00006019357330019A2B367D7016384071AF8
:105FD0009387F5FF638A073A638BC523BE8591B526
:105FE0006398051C9386140093F7E67FC1EFB367AF
:105FF000E301639F0434638C0744B367D701639361
:1060000007460E051318D3010D813368A800935776
:1060100033006DA8B385984063960420B367E3010D
:10602000638C07309387F5FF638807401305F07F83
:106030006382A520BE859307800363C1B72AFD470D
:1060400063C7B73C930700028D8F3318F3003356B4
:10605000BF00B317FF003368C800B339F0003353F3
:10606000B3003368380133076740ADACB367D7017D
:10607000638207109387F5FF638E071E638FC52D1C
:10608000BE85D1B59307F07F638BF606FA9E33B6D3
:10609000EE01B307E300B2971398F70193DE1E00F9
:1060A000B369D80113D61700B68493F77900E39F3C
:1060B00007E09317D60113D839003368F800A68596
:1060C000935736001307F07F6380E506B207B1836C
:1060D00013F7F57F05883DBD3367D7013338E000FE
:1060E000B309E801B3B7E901338667009317860067
:1060F000E3DD07FA85049307F07F639BF4180588B6
:106100001307F07F8147014831B5639007106300A2
:10611000083C131836009317D7011358380033681A
:10612000F800368493573700B367F800E9DB014481
:106130001307F07FB70708000148E9BB370680FF67
:106140007D167D8E93F77900998CE39107D895B7EA
:106150004E85E12913078501FD47E3D3E7D21306F6
:1061600085FFB397C900814935B33368D701333808
:106170000001D5B1131835009317D3011358380017
:106180003368F8009357330035BFB309DF41330953
:10619000E34033363F013309C9409317890063CA8E
:1061A000072033E82901E31708CC8147014439BFB0
:1061B000B385984063810414B70680009307F07F8D
:1061C0003363D3006381F8209307800363CCB72245
:1061D000FD4763C9B72C930700028D8F3318F30076
:1061E000B356BF00B317FF003368D800B339F000CF
:1061F0003353B300336838011A97B309D801B3B7E2
:10620000D9013386E700C684D5B5E31208F2131826
:1062100035009317D301135838003368F8009357AB
:10622000330019B7370580009307F07F3363A3006D
:10623000E393F8E00E061318D7010D823368C80007
:10624000935737003684CDB505179306000233D730
:10625000E700630AD600930600043386C6403396EF
:10626000C700B3E9C90033383001B369E80001461B
:10627000814425BDB309DF01B307E30033BFE90162
:106280003386E701931786008544E3D007E289440B
:10629000B70780FFFD17F18F13D7190013F8190006
:1062A000336807019399F701B3E9090113D6170081
:1062B00019B9138805FE93070002B3590701638AD1
:1062C000F50093070004B385B7403317B700B3EE6A
:1062D000EE003338D00133683801B5BE3363E301D3
:1062E00033386000B3890E41B3B73E013306F7403F
:1062F000C6843684BDB6B367E30163870718938706
:10630000F5FF638C071C9306F07F638ED50ABE856C
:1063100065BD930700028D8FB3D9BE003318F70017
:10632000B39EFE00336838013357B700B339D0014C
:10633000336838013A936DB3131836009317D701B9
:106340001358380033E807013684935737009DBB54
:10635000BDCB3367D701E31C07DC0E051318D3014F
:106360000D813368A800935733007DBBE30F08E22B
:10637000131836009317D701135838003368F80004
:1063800036849357370099B3B309DF41B307E3402D
:10639000333F3F013386E7418544E1B413183500AC
:1063A0009316D3011358380033E80601935733008E
:1063B000A5BBB389EE413306674033B93E013309CB
:1063C0002641368445BC0E061318D7010D8233686A
:1063D000C8009357370089BBB309DF41B307E340D7
:1063E00033363F013386C7409317860063D7070AC9
:1063F000B389EE41B3076740B3BE3E013386D74150
:106400003684D1B43363E30133386000FDB31388BD
:1064100005FE93070002B3590301638AF500930751
:106420000004B385B7403313B300336F6F003338C4
:10643000E001336838017DB5B389EE41B3076740A9
:10644000B3BE3E013386D7413684854419BC131848
:1064500036009317D701135838003368F800935764
:106460003700ADB1B309DF01B307E30033BFE90182
:106470003386E70193178600E3D907C2B70780FF89
:10648000FD177D8E854415B10E061318D7010D82B8
:106490003368C8009357370035B133E8C900E306C5
:1064A00008D021B1138805FE93070002B3590301F8
:1064B000638AF50093070004B385B7403313B30034
:1064C000336F6F003338E001336838013DB3014466
:1064D0001307F07FB707080035BCB309DF01B30726
:1064E000E300B3BED9013386D70169BB93D7450119
:1064F000B70610001387F6FF93F7F77F1306E03F08
:106500006D8FFD81635CF6001306D041635AF6007F
:10651000370500801345F5FF2E9582800145828066
:10652000130630431D8E7D48558F635DC80093066A
:106530003041B387F640B357F7003305F040E5F13B
:106540003E8582809387D7BEB317F7003355C500C9
:10655000C98FE5B7411106C622C426C205CD93579F
:10656000F541B3C4A7009D8C2A8426857D28930617
:10657000E041898EA9477D8093F6F67F63CDA7021F
:106580002D47098FB3D7E4005505B207B394A40093
:10659000B18329A00144814681478144B207D206D4
:1065A000B1837E04D58FC18FB24022442685BE853B
:1065B0009244410182805515B397A400B207B1837C
:1065C0008144E9BF15CD411122C406C62A84B128F1
:1065D0009306E041898EA94793F6F67F63DCA70214
:1065E0005515B317A400B207B1830147B240224446
:1065F000B207D206B183D58F3A85BE85410182802C
:1066000081478146B207D206B1830147D58F3A85CB
:10661000BE8582802D47098FB357E400B207130768
:1066200055013317E400B183D1B7C167637EF5022A
:106630009307F00F1307000263ECA70097670000B1
:10664000938747F5AA9703C507003305A7408280C3
:106650002181976700009387E7F3AA9703C5070096
:1066600061473305A7408280B7070001636EF500DC
:106670006181976700009387E7F1AA9703C5070038
:1066800021473305A74082804181976700009387A7
:1066900067F0AA9703C5070041473305A7408280EA
:1066A0009387C1829C434111328806C6AA882E87EF
:1066B000C8473686976700009387C7FD63170800B1
:1066C000976700009387C79E3E88C686976500003F
:1066D000938545FD1920EF206066397132D436D696
:1066E0003EDA3AD842DC46DE9387C1822E86AA85FE
:1066F0008843341006CE36C6712AF240216182806A
:1067000001476314E60001458280B307E5000507F1
:10671000B386E50083C7070083C6F6FFE383D7FE91
:106720003385D7408280B3C7A5008D8B3307C50062
:1067300081E78D4763EEC700AA876370E50A83C6C9
:10674000050085078505A38FD7FEE3EAE7FE828073
:1067500093763500AA8791CA83C60500850785050B
:10676000A38FD7FE93F63700FDB79376C7FF138646
:1067700006FE63F0C70683A3050083A2450083AF2E
:10678000850003AFC50083AE050103AE450103A339
:10679000850183A8C5019385450223A0770003A83E
:1067A000C5FF23A2570023A4F70123A6E70123A8CE
:1067B000D70123AAC70123AC670023AE1701938733
:1067C000470223AE07FF75B790419107910523AEAD
:1067D000C7FEE3EBD7FEE3E4E7F6828063F3A504AC
:1067E000B386C500637FD5029345F6FF8147FD1749
:1067F0006393F50082803387F600034807003387F0
:10680000C7002A9723000701DDB73387F5008346C9
:1068100007003307F50085072300D700E317F6FECE
:1068200082808147E5BF1C46FD171CC663DA07005E
:10683000184E63C5E700A9476394F5006F208032C6
:106840001C422E851387170018C22380B700828050
:10685000011122CC26CA4AC84EC652C406CE2A8985
:10686000AE893284B304D6007D5A63149400014586
:1068700011A8834504004E864A85EFF0DFFA05042F
:10688000E31545FFF2406244D2444249B249224AEC
:1068900005618280357122CD26CB4AC94EC706CF0D
:1068A00052C556C35AC1DEDEE2DCE6DAAA89AE84FE
:1068B0003289368409C51C4D99E3EF30C04497678F
:1068C00000009387A7F8639DF40C83A4490083D745
:1068D000C400A18BE5CB9C48F5C793070002A30435
:1068E000F1029307000302D22305F10222C6930BA3
:1068F0005002976A0000938AEADD054C294B4A84CE
:106900008347040099C36392770FB30C2441638ECD
:106910000C00E6864A86A6854E85EFF07FF3FD578C
:106920006306F51E9256E69636D283470400638FBF
:10693000071CFD571309140002C802CE3ECA02CC40
:10694000A309010482D48345090015465685EF301A
:10695000705D13041900C24759E913F7070109C70D
:1069600013070002A309E10413F7870009C71307FF
:10697000B002A309E104834609001307A002638063
:10698000E608F2474A8481462546034704009305FA
:106990001400130707FD6379E60AB5CA3ECE85A841
:1069A00097670000938787EC6395F40083A48900C0
:1069B00039BF97670000938767E7E39AF4F083A4F1
:1069C000C90031B7A6854E85EF20202619D57D5503
:1069D000FA406A44DA444A49BA492A4A9A4A0A4B6E
:1069E000F65B665CD65C0D618280050411BF3305E1
:1069F00055413315AC00C98F3EC82289A9B732472B
:106A000093064700184336C6634907023ACE034748
:106A100004009307E002631FF70403471400930781
:106A2000A002631BF702B2470904138747009C4387
:106A30003AC663C107023ECA35A83307E04093E770
:106A400027003ACE3EC8E1B7B387670385462E8458
:106A5000BA9725BFFD57C5B7050402CA81468147CD
:106A600025460347040093051400130707FD6378C8
:106A7000E606F1F2834504000D4617650000130594
:106A8000E5C5EF30304A11CD97670000938707C501
:106A90001D8D93070004B397A700424505045D8D43
:106AA0002AC883450400194617650000130545C32D
:106AB000130914002304B102EF30D04625C1970713
:106AC00000009387C71E95E74247B2471377071028
:106AD00009CF91073EC69257D2973ED20DB5B387E4
:106AE000670385462E84BA97ADBF9D07E19BA1073A
:106AF000D5B77800970600009386C6D526860C0881
:106B00004E856522FD572A8AE317F5FC83D7C4001A
:106B100093F70704E39D07EA12555DBD78009706D9
:106B20000000938626D326860C084E85B927D9BF48
:106B3000797122D44AD052CC56CA5AC806D626D227
:106B40004ECE3A8AAE8A32843689428B01476358E8
:106B50000600370700803344C7001307D0022380A4
:106B6000E70093F4F8FD930760048D466388F40012
:106B70009307500489466393F4000509DA87930864
:106B8000C100130881004A87D6852286EF20A02FF6
:106B900093077004AA896396F400137A1A00630AB3
:106BA0000A0493076004338A29016397F40203C738
:106BB000090093070003631EF700014681465685CE
:106BC000A285EFE0BFB611C5854733892741232051
:106BD0002B0183270B003E9A014681465685A285EC
:106BE000EFE0DFB411E152C613070003B24763E2DE
:106BF0004703B2474257B2502254B38737411CC3B0
:106C00004E8592540259F249624AD24A424B45613A
:106C100082809386170036C62380E700C1BF230019
:106C2000C500130725009307B00263D60500B3051E
:106C3000B0409307D002A300F500A54763DAB7047C
:106C400041119307F100BE88294813033006B3E6CB
:106C500005031386F7FF93860603A38FD7FEB3C6FB
:106C60000503634DB30093860603F917A30FD6FE01
:106C700063E917013305A74041018280B287B685D9
:106C8000F9B7850783C6F7FF0507A30FD7FECDB772
:106C90009307000313074500938505032301F500BF
:106CA000A301B5003305A740828019713ACE86DE74
:106CB000A2DCA6DA2E84CAD8CED6D2D4B689DAD04F
:106CC000DECEE2CC3289D6D2E6CAEAC8EEC6AA84C3
:106CD000EF30B00F832B05005E85EF00B078032BFB
:106CE0000400724702DC93760B102A8C034A84015D
:106CF0001C43F1CA9386470014C39C430810984371
:106D00003AD0D8433AD298473AD4DC473ED6EF50EF
:106D1000400728C46CC4832CC40417670000130701
:106D2000E79C832A8404032D0700832D4700939753
:106D30001C0085836A86EE865685BE853ECEEF4072
:106D4000F04941EDF2476A86EE865685BE85EFE052
:106D50007FAF6354A008014681465685E685EFE083
:106D60007FAE635605009307D002A301F404930796
:106D70007004976A0000938AEA9763F64701976A5E
:106D80000000938A6A97137BBBFF8D472320640121
:106D90001CC8014B4E87CA867018A2852685C12E55
:106DA000FD5C631E95157D55F6506654D6544659C4
:106DB000B659265A965A065BF64B664CD64C464D4B
:106DC000B64D096182809D07E19B9386870014C3BD
:106DD0009843DC4338C47CC43DBF5686E68656855E
:106DE000E685EF40B03F11CD93077004976A00002D
:106DF000938ACA90E3F947F9975A0000938A8A6CFC
:106E000059B75C407D57137DFA0D6395E7089947A4
:106E10005CC0544013670B403C18D6853EC018C078
:106E20009307310302C2D288130841036686268580
:106E3000EFF01FD093077004AA8AD255631BFD00A0
:106E4000F55763C5F5005C4063D8B708791A137A23
:106E5000FA0F9307500663E64705FD1552861305A2
:106E600004052EDAEFF0BFDB625785462A8BB307A5
:106E7000A7001CC863C5E6001840058B19C3850729
:106E80001CC883473103E38707F09307D002A301AF
:106E9000F40409B713077004E31DEDF6BDFB854745
:106EA00085BF93076006631BFA025C40635BB0001A
:106EB0000CC881E71840058B09CF8507AE971CC821
:106EC00009A889E718408546058B19C393862700D2
:106ED00014C82CCC014B75B7130A7006E25763C96E
:106EE000F5001C400CC8858BEDD793871500C1BFFA
:106EF00005476344B00009470D8FBA97C9B71C40D6
:106F000013F7074015E314485686CA8526858299EB
:106F1000E30B95E91C40898B63960724F25748449C
:106F2000E354F5E83E8549B513075006637B4719DE
:106F300028446C4401468146EFE04FFF39E985461D
:106F4000175600001306C67BCA8526858299E30C76
:106F500095E55257E2576345F7001C40858BDDDB12
:106F6000E2865E86CA8526858299FD57E30DF5E2A5
:106F7000014A930AA4017D5BE257FD17E35CFAF82E
:106F800085465686CA8526858299E30E65E1050AFF
:106F9000E5B7D2576346F00685461756000013063C
:106FA0002676CA8526858299E30F95DFD2576257E8
:106FB000D98F81E71C40858BB1DFE2865E86CA856A
:106FC00026858299FD57E300F5DE014A130BA401E3
:106FD000FD5BD257B307F040634BFA00E25656868A
:106FE000CA8526858299FD57E316F5F26DBB854665
:106FF0005A86CA8526858299E30775DB050AD1BFC3
:107000003C4C625A63D347013E8A635A4001D286A0
:107010005686CA8526858299FD57E306F5D8814CA8
:10702000130DA401FD5D09A885466A86CA852685DB
:107030008299E30AB5D7850C032B8405D287635365
:107040000A008147B307FB40E3C0FCFE5257E257FA
:10705000634DF7021C40858B8DEBE2575257338A04
:10706000E7406344EB00338A6741635B4001D286AB
:1070700033866A01CA8526858299FD57E305F5D2D4
:10708000814A130BA401FD5B15A0E2865E86CA85CA
:1070900026858299FD57E312F5FC31B385465A8661
:1070A000CA8526858299E30075D1850A5257E25731
:1070B000998F528763530A000147998FE3C0FAFE04
:1070C00091BDE25605476344D700858BB5C7854619
:1070D0005686CA85268582997D5AE30645CDE28685
:1070E0005E86CA8526858299E30F45CB28446C4489
:1070F00001468146EFE08FE31DC9E25613861A0070
:10710000CA85FD1626858299E30F45C9DA861306DE
:107110000405F9B585465686CA8526858299E30415
:1071200075C9050AE257FD17E346FAFEC5B7014ADD
:10713000930AA401FD5BFDB785465686CA85268560
:107140008299E31595FD85B185465686CA852685C3
:107150008299E30A65C5050A5C447257998FE34535
:10716000FAFE6DBB014A930A94017D5BF5B7797114
:1071700056CA9C49BA8A984522D426D24ECE52CCC1
:1071800006D64AD05AC85EC6AA892E84B284368AE8
:1071900063D3E700BA879CC00347340419C385074B
:1071A0009CC01C4093F7070281C79C4089079CC084
:1071B0000329040013796900631A0900130B940171
:1071C000FD5B5C449840998F634CF9041C408346F6
:1071D000340493F70702B336D000A5EB130634044A
:1071E000D2854E85829AFD576303F5041C401146F3
:1071F0009840998B544481446397C700B384E64018
:1072000063D3040081441C4418486354F700998FE9
:10721000BE94014969047D5B63982405014509A872
:1072200085465A86D2854E85829A631E75017D55A4
:10723000B250225492540259F249624AD24A424B05
:10724000B24B456182800509ADBF3307D4001306F8
:107250000003A301C7040347540493871600A297B1
:107260008906A381E7049DBF85462286D2854E8587
:10727000829AE30E65FB050945B7797122D426D2BF
:107280004AD04ECE06D652CC56CA5AC8B68983C604
:107290008501930790063289AA842E8413863504CB
:1072A000638DF60263E2D706930780056389F618BB
:1072B00063EDD7006382062293073004638FF60ADA
:1072C000930A24042301D404D1A0930730066386D3
:1072D000F60A93074006E395F6FE1C40084393F632
:1072E000070893054500CDC61C410CC363D80700B1
:1072F0001307D002B307F040A301E404975600003F
:1073000093864640294775A8930700076385F616BC
:1073100063E5D7029307E006638CF6189307F0063F
:10732000E390F6FA0C401C4313F805081385470058
:107330006308080608C39C4395A893075007E38396
:10734000F6FE93078007638CF61293073007E399E4
:10735000F6F61C43D04181459386470014C383AAA7
:1073600007005685EF30003C01C53305554148C044
:107370005C401CC8A301040471A81C43930A2404A4
:10738000938647009C4314C32301F4048547D5B773
:1073900093F607041C410CC3B1DAC207C187B9B721
:1073A00093F5050408C3C1D983D707001307F00676
:1073B0006388E60E975600009386C6342947A301DA
:1073C00004044C400CC463C5050008406D9908C016
:1073D00099E3B28A91CDB28AB3F5E702FD1AB69568
:1073E00083C505002380BA00B3D5E70263F0E70C3C
:1073F000A147631EF7001C40858B91CB58401C4869
:1074000063C7E70093070003A38FFAFEFD1A330654
:10741000564110C84E87CA867000A2852685EFF0B7
:107420001FD57D5A631E450B7D55B2502254925490
:107430000259F249624AD24A424B45618280A38294
:10744000D504975600009386E62B0C40084313F8AA
:1074500005081C411105630D080208C313F7150048
:1074600001C793E505020CC04147B1FB0C4093F501
:10747000F5FD0CC0A9B79C4193E707029CC1930797
:107480008007A302F404975600009386E62875BF90
:1074900013F8050408C3E30308FCC207C1837DBFDA
:1074A0009756000093860626214711BFAE872DB759
:1074B00094411C43CC4913F8060813854700630622
:1074C000080008C39C438CC301A808C393F60604B4
:1074D0009C43F5DA2390B70023280400B28A1DBF2D
:1074E00014485686CA8526858299E30F45F31C40C9
:1074F000898B8DE7B2474844E359F5F23E8535B7AD
:1075000085465686CA8526858299E30F65F1050A68
:107510005C443247998FE345FAFEE9BF014A930A7A
:1075200094017D5BF5B79C451D71A2CCCEC6DAC037
:1075300066DA86CEB28CA6CACAC8D2C4D6C25EDE0D
:1075400062DC6AD86ED61386F7FF1307C015368B38
:10755000AA892E8481466377C700938637EA93070A
:10756000D0159CC51C40930AC401D68493E70778C4
:107570001CC00149814D014C014A014D814B13064C
:107580009004130800708548930E00400943130EC1
:1075900050061D4F18441DCB83A70C0083C707005E
:1075A000638BC7126368F60C9305900363E4F50AD6
:1075B0009305100363FBB7149305D0026383B716DA
:1075C00063E3F5041307B002638DE71463060D004F
:1075D0001C4093F7F7EF1CC0FD1D854763EBB721F7
:1075E00063ED9A1E0549F64066444A85D6444649ED
:1075F000B649264A964A064BF25B625CD25C425D13
:10760000B25D256182809305E002638FB714930514
:107610000003E39DB7FA0C4013F505107DC593F503
:10762000F5F70CC0050D81C60507FD1618C41C44EE
:10763000FD171CC41C4885071CC883A74C00FD17F8
:1076400023A2FC006356F01683A70C00850723A035
:10765000FC0089B7130750046382E7121307600424
:10766000638BE70E13071004E392E7F6E3901DF730
:10767000894D65A06384C7116361FE04130740054B
:10768000638FE70C6364F7021307E004E390E7F409
:1076900063910D0A63110D0A184093750770639C7E
:1076A00005091377F78718C0854D85A8130790053E
:1076B0006389E7041307100645BF1307E006E38953
:1076C000E7FC6368F702130760066386E7081307A1
:1076D0009006E39DE7EE63190906E31B0DEE1840E3
:1076E00093750770E39A05EF1377F78718C005497C
:1076F0002DA0130740076384E70613079007E3975D
:10770000E7ECE315E9ED214909A833872D01E31FD3
:1077100007EA18401377F7E718C02380F4008504C0
:1077200039B7184093750708E38205EA1377F7F72E
:10773000E5B7638D6D06630519011147E318E9E8A4
:1077400005091379F90FD1BF1307D9FF1377D70FA5
:10775000E31E07E6F5B7E31B69E60D497DBF194750
:10776000E316E9E61D4955BF184093750720E38FDE
:1077700005E41377F7D718C0EA8B45B7184093751F
:1077800007506388D50193750740E38105E4E3055D
:107790000DE49375072081E5330A7D41268C13772C
:1077A000F7871367071818C0014D85BF8D4DB5B712
:1077B00083270418E6854E8536C68297B24613069F
:1077C0009004130800708548930E00400943130E7F
:1077D00050061D4FE30005DCD5BBFD148327C417FD
:1077E00083C5040066864E8582971C48FD171CC819
:1077F000C5BB9307F9FF19476366F7028947A68D52
:1078000063F12709330799401377F70F8D46B38744
:10781000ED0093F7F70F63ECF60275191379F90F82
:10782000B38424411C4013F7071045C393F7074066
:10783000A1CFE3F99ADAFD148327C41783C50400A6
:1078400066864E8582971C48FD171CC8DDB7FD1D56
:107850008327C41783C50D0066864E853AC6829776
:107860001C488D463247FD171CC855B7FD148327A9
:10787000C41783C5040066864E8582971C48FD1791
:107880001CC8E3E59AFEB9BB1C4883C5F4FF138905
:10789000F4FFFD171CC8930750066382F502930797
:1078A0005004638EF5008327C41766864E85829741
:1078B0001C4883C5E4FF1389E4FFFD171CC8832718
:1078C000C41766864E858297CA84032904001379FB
:1078D00009016313090C238004001C4013070040B6
:1078E00093F70760639EE7023386AB416396AB056F
:1078F000D68501464E85EF10000718402A8AAE8AC9
:107900009376270083270B00A9C6138747002320FF
:10791000EB009C4388C3CCC35C4485075CC4E1B1E5
:10792000E3080AFC0146A94693051C004E85EF10AA
:10793000E01A33064541E2849307F41663E4F40049
:107940009304E41697550000938545DE2685C12CE7
:1079500045B7938647002320DB00118B844319CF62
:10796000AA8556860808EF40E010D2466247F247E3
:107970004246D4C098C490C0DCC479BF2A86AE8683
:10798000EF40C00509C50145292C88C071B7528553
:10799000D685EF406028D5BF0149B1B139713EDAD3
:1079A0002ED232D436D63AD842DC46DE9387C18214
:1079B00022CC804326CA06CEAA8411C41C4C81E77F
:1079C0002285EF2040340C4454102686228536C68A
:1079D000EFE05FECF2406244D24421618280011109
:1079E0009387C18222CC804306CEAA8501C81C4C55
:1079F00091E72AC62285EF200031B2451044228546
:107A00006244F24005616F30B042011126CA4AC893
:107A100006CE22CC4EC652C4AA842E8909C51C4D5E
:107A200099E3EF20402E9C4C804481E72685EF208F
:107A3000802D97570000938767E1631DF402C040D3
:107A40008357C400A18BB9C71C48A9C7FD59294A4F
:107A50001C4483450900FD17A1ED1CC463D1070830
:107A60002286A9452685EF10E00FFD576309F50230
:107A700029453DA097570000938747DF6314F40022
:107A800080447DBF97570000938747DAE31AF4FAE2
:107A9000C0447DB7A2852685EF10201945D97D55B4
:107AA000F2406244D2444249B249224A056182808E
:107AB0001CC4050963D70700184C63CBE700638932
:107AC00045011C401387170018C02380B70049B731
:107AD00022862685EF100009E31C35F7C9B71C4044
:107AE0001387170018C029472380E70051B79387F1
:107AF000C182AA8588436FF05FF113D745414111D8
:107B00001377F77F06C6930617C04D4E2A88AE87B7
:107B1000AE886342DE0663DD0600370700808146DB
:107B20006D8F14C258C2B2404285BE854101828029
:107B3000370710007D173357D740B3F6E50033E31E
:107B4000A600631B03005CC2B70700802320060168
:107B5000B3F7F8000148C1BF1347F7FF0148B377F7
:107B6000B700232006015CC2BE864286EFE06FA408
:107B70002A88AE874DBF130E3003E346DEFC930622
:107B8000D7BE7D573357D700B376A700CDDE134756
:107B9000F7FFB378A700232016014CC2AE864686B5
:107BA000F1B7975700009387E7B888438280357113
:107BB0003ECBA6DA36C73AC942CD46CF9387C182BB
:107BC00086DEA2DC844363DB05009307B0089CC01B
:107BD0007D55F6506654D6540D61828093078020FF
:107BE000231AF1002AC42ACC814799C19387F5FF53
:107BF0003EC83ECE7401FD572E8426852C00231BE3
:107C0000F10036C2EF30E07AFD576355F500930777
:107C1000B0089CC05DDCA247238007005DBF3571C2
:107C20003ECBB707008093C7F7FF3ECE3EC8C17773
:107C30009387872032C536C73AC942CD46CF3ECA60
:107C40009387C1822AC42ACC884334012E862C0013
:107C500086DE36C2EF30E075A24723800700F6507B
:107C60000D618280AA87850703C7F7FF6DFF338503
:107C7000A7407D158280AA8709CA850503C7F5FF3D
:107C800085077D16A38FE7FE65FB3E966393C700CD
:107C900082808507A38F07FED5BF011122CC2A87DA
:107CA0002E843A85A28532C606CEEF3020163246A3
:107CB0002A88AE8805C651801374F47F9307B006F6
:107CC000818F635DF000D2073707F03F01483E9790
:107CD0004286BA86EFD07FC22A88AE88F2406244DC
:107CE0004285C6850561828035714AC92A893685F3
:107CF00032D436C606CF22CD26CB4EC7EAD8EED632
:107D00002E8D52C556C35AC1DEDEE2DCE6DA82C8E9
:107D1000EF20500BAA8D084181440144EFF09FF4FD
:107D2000B246AA89EAC635469305B0021305D002C9
:107D300013080002A548B64703C70700636BE608AF
:107D4000637F17095DC702C8364A93070003814A5B
:107D500003470A00631DF71283471A0013078005C3
:107D60006388E70013068007130700036397C710B3
:107D7000C24736889808D40817560000130686A113
:107D8000EC004A85EF20001B93797500AA8A63886E
:107D9000090099476398F906050AD2C602C8A25796
:107DA00081C7B64722571CC3C247A1CBB705008085
:107DB000A18DFA406A4426854A49DA44BA492A4ADA
:107DC0009A4A0A4BF65B665CD65C465DB65D0D6111
:107DD00082806309B7006304A702E31607F78507EB
:107DE000BEC691BF02C813871700BAC683C7170063
:107DF000A1FFA257EAC602C8CDF7A2855DBF05471D
:107E00003AC8D5B7464611CA93055003A808EF30C3
:107E10000024C6454A85EF20501BFD19914763EEAB
:107E2000370117570000130727918A09BA9983A7CA
:107E30000900BA978287E644764493FA8A00E38081
:107E40000AF6B70700805D8C99BFF6453704F0FF4E
:107E50007D14B3F785005644E64413043443931568
:107E6000440133E4B700D1BF3704F07FF9B7B70559
:107E7000008013C4F5FFFD54C9B7B64793861700B9
:107E8000B6C683C71700E38AE7FE91DB854AB64C86
:107E9000014A814B014CA546A145A9473645034BF4
:107EA000050013070BFD1376F70F63FDC60483A5CA
:107EB0000D004E86EF3050193DC1DA87E28D8146C4
:107EC000014B0145130750066387E7001307500471
:107ED00081496399E71663960D00B3E7560191DB7C
:107EE000814D364D1307B00293071D00BEC6834770
:107EF0001D006382E70E1307D00201486393E70E6B
:107F00000548D9A863C98501B38BFB02BA9B050557
:107F1000050CAAC661B7330AFA023A9ACDBF3645B4
:107F200081464E95AAC683470500630D0C06014B9A
:107F3000E28D138707FD25466376E602054559B7AE
:107F4000B647850613861700B2C683C71700E389B4
:107F5000E7FE1387F7FC2146E36AE61EB64C368B34
:107F6000814D8146938707FD1387160085C73A9B8D
:107F70003385B6016E872148C14829466317A70299
:107F8000850DB69DA14663CFE6022947B38BEB0270
:107F90000147BE9BB64793861700B6C683C7170036
:107FA000BA8641BF130700035DB793051700634608
:107FB000E800B38BCB022E87D1B7E3CEB8FE330AED
:107FC000CA02D5BFC1460147E3C6B6FDA946330A7A
:107FD000DA023E9AC1B7014893072D00BEC6834717
:107FE0002D00138707FD25466367E60C1307000382
:107FF0006386E70A1387F7FC214681496364E60438
:10800000B648138707FD2543294EB6471386170048
:10801000B2C683C71700938507FD93F5F50F637606
:10802000B3089569330616419389F9E1A148CE85D5
:1080300063C6C800BA8963D3E500AE89630408004B
:10804000B309304163980D0CB3E6DA00E39906D426
:10805000E31105DA1307E004638AE7066340F706D5
:1080600013079004E397E7D897450000938585713F
:10807000E800EF20C03BE30E05D6B6479745000069
:1080800093858570E800FD17BEC6EF20403A01E5F4
:10809000B6478507BEC63704F07F11B3B6471386CF
:1080A0001700B2C683C71700A1B73307C703BA9733
:1080B000138707FD99BFEAC6814969B71307900680
:1080C000E384E7FA1307E006E395E7D2974500005B
:1080D0009385056CE800EF208035E30C05D0B647AA
:1080E00003C70700930780026313F702B0089745A0
:1080F00000009385656BE800EF20603695476318B4
:10810000F500F6453704F07FE6444D8C49B9370455
:10811000F8FF71B1B38A694163130C006E8CC147DB
:108120006E8D63D3B701414D5E85EFE0AFC9A547C2
:10813000AA842E8463DCB70393077DFF139737006F
:108140009747000093870778BA979043D443EFD0BE
:10815000CFFA2A845285AE84EFE0CFC62A86AE8657
:108160002285A685EFC05F8EAA842E84BD4763CD8D
:10817000B709E3860AC2635450075947634357035C
:108180008E0A974700009387E773BE9A03A50A00FB
:1081900083A54A002686A286EFD02FF6AA842E84D5
:1081A000FDBE130750023307B741634F5705B38D28
:1081B000B741174900001309E97093973D00CA972A
:1081C0008843CC43B38DBA412686A2868E0DEFD06C
:1081D000CFF2CA9D03A60D0083A64D0075BFA95717
:1081E00063C4FA02B3093B41139B3900974900006D
:1081F0009389496DDA9903A6090083A6490026856B
:10820000A285EFC07FF759BF338DAD41569D6357AF
:10821000A0119377FD0099CF174700001307876AD5
:108220008E07BA978843CC432686A286EFD0EFEC20
:10823000AA842E84137D0DFF63080D0A9307401353
:1082400063D5A705014B814902C6814B93072002E4
:108250002320F9003704F07F8144B247E38107B45B
:10826000C6454A85EF206056DE854A85EF20E055F9
:10827000CE854A85EF206055B2454A85EF20E0540F
:10828000DA854A85EF20605419BE135D4D4026857E
:10829000A2858147014A05489748000093880860F5
:1082A0006346A80599C3AA842E84174700001307C4
:1082B000E75E93173A00BA978843CC433707B0FC80
:1082C00022972686BA86EFD04FE33704F07FB37744
:1082D000B4003707A07CAA84E366F7F63707907CE2
:1082E000637AF7027D14FD54014ADDA813771D005F
:1082F00011CF13173A00469710435443EFD0EFDFE6
:10830000854705489748000093884859050A135D3A
:108310001D4079B7370450032E94F9B7E3060DFCDE
:10832000330DA0419377FD0099CF17470000130745
:1083300067598E07BA979043D4432685A285EFC02C
:10834000BFE3AA842E84135D4D40E30F0DF8FD4773
:1083500063DDA701014B814902C6814B93072002CF
:10836000814401442320F900CDBD137A0D0163043B
:108370000A00130AA0062685A28597470000938766
:10838000E743014793761D0081CA9043D4433EC61C
:10839000EFD0AFD6B2470547135D1D40A107E313E9
:1083A0000DFE19C3AA842E8463050A029357440163
:1083B00013F7F77F9307B006998F635CF0007D4752
:1083C0006354F7221307400381446359F7203704AD
:1083D0007003014681462685A285EFD02FB53DD991
:1083E0005E87EE866286E6854A85EF20C04B2AC608
:1083F000E30A05E493D7FA41B3093B41B3F7F90027
:108400003ED056CE63D30A0002CEB247014B81491B
:10841000B1073ED8B7071000FD173ED6B2474A85D0
:10842000CC43EF20C031AA8BE30205E2B247C2552C
:108430003105904B09060A06EFE0EFAEB808D40804
:108440002286A6854A8526CA22CCEF20D02BAAC830
:10845000E30E05DE85454A85EF20405AAA89E307E9
:1084600005DED64763C707180257724C338DE70005
:108470006647B387474193066003BA97FD17930D8C
:1084800020C0998E63D6B7193387FD407D46998EFB
:108490006346E616854DB397ED003ED2814C369C7F
:1084A000B30DDD00529CEA8763D3AD01EE876353C1
:1084B000FC00E2876358F000B38DFD40330CFC40B4
:1084C000330DFD4082576358F002CE853E864A85C3
:1084D000EF20C068AA89E30B05D64646AA854A85DF
:1084E000EF2080532ADAE30305D6C6454A85EF20FC
:1084F000C02DD257BEC8634FB011635A50017246A7
:10850000DE854A85EF208065AA8BE30105D4635A96
:108510008001DE8562864A85EF202070AA8BE30702
:1085200005D2635AA001CE856A864A85EF20E06EA7
:10853000AA89E30D05D0C6455E864A85EF20E07D19
:108540002A8BE30505D0032CC500CE852326050024
:10855000EF2080796359050C336C9C0063110C1279
:108560009317C400639D0710B707F07FE18F3707AB
:10857000B0066376F71083274B0191E703270B01C1
:10858000854763DEE70EDA8505464A85EF20E06819
:10859000CE852A8BEF2040756353A00E630C0A1022
:1085A000B707F07FE18F3707B0066345F71037074D
:1085B0007003E355F7DA0147B70750392685A285DE
:1085C0003A86BE86EFD06FB32E84C98DAA84E39914
:1085D00005C8930720022320F90059B181177D5760
:1085E000B317F7007D8CF5B37D57B317F700FD8CFB
:1085F000CDB37247025D330CF7409DBD930C20BE96
:10860000B387FC40854CB39CFC0085473ED241BDFE
:10861000814CE5BFC6456E864A85EF200060AAC83A
:10862000E31D05EC25B169E9370710007D17B37725
:10863000E40063090C046399E7047D5763000A02B0
:10864000B707F07FE18FB706A00663E9F600D18394
:108650009306B006B387F6403317F7006396E4023B
:10866000B707F07FFD176315F400FD57E380F4BEF4
:10867000B705F07FE18D370410002E948144E31C90
:108680000AF2F9BEC58F99DB63820C04B3FC8C003F
:10869000E3870CFE52862685A285630F0C02EFF05D
:1086A000CFDF2A86AE865245E245EFC0EFB9AA84F5
:1086B0002E84F1B7B705F07FE18D3704F0FFA29566
:1086C000370410007D144D8CFD5455BF9257B3FDF7
:1086D0009700E3860DFA7DBFEFF02FDC2A86AE8689
:1086E0005245E245EFD0EFEC01468146AA842E8444
:1086F000EFD0CF8349F59DB1CE855A85EF20F00D9F
:1087000097470000938787059043D4432A8DAE8D09
:10871000EFD04F936342A01063010C0A814D370DD7
:10872000F03F0147B707F03FB706F07FB37CD400B6
:10873000B706E07F639FDC166AD2370DB0FC229D3E
:108740002685EA853EDE3ADC6EDAEF20206CD258D0
:1087500012582A86AE864685C285EFD00F9A2686A5
:10876000EA86EFC06FAEAA843705F07F3376B50096
:10877000B706A07C6257F2576365D60C6247930731
:10878000F5FF6396E7005247FD57E381E7ACB70773
:10879000F07F1384F7FFFD54C6454A85EF20E002C1
:1087A000DE854A85EF206002CE854A85EF20E00114
:1087B000DA854A85EF20600195B1B1E0B257E18FCB
:1087C000A1E7974700009387E7F89043D4436A8571
:1087D000EE85EFD02F87634D050297470000938702
:1087E000E7F69043D4436A85EE85EFD00F912A8750
:1087F000AE87370D0080BA8D334DFD0035B7854704
:108800006394F400E30C04B4814D370DF0BF11BF45
:108810000147B707E03FF1BF97470000938707F391
:108820009043D4436A85EE85EFD02F8D2A87AE879B
:108830002E8D63160C00370D0080334DBD00AA8DC0
:10884000E5B5370450032E94E3180AF4B706F07F19
:10885000E18EE393DCF4BE853A853A8DBE8CEFD091
:10886000FFC8EFD03FCF2A86AE866A85E685EFD077
:108870004FD4B2572A8DAE8DE18FC58F33EC87016F
:10888000630B0C0A97470000938747EE9043D4434D
:10889000EFC05FFBE346059C97470000938787ED99
:1088A0009043D4436A85EE85EFC0FFEEE356A0EE19
:1088B00045BA630D0A04B706A00663E99605974614
:1088C0000000938626EA9042D4423A85BE853ADA81
:1088D0003ED2EFC03FF7925752576344A0023A8509
:1088E000BE85EF30601311E10545EFD0BFCD2A877B
:1088F000AE872E8D63160C00370D0080334DBD0002
:10890000AA8DB705B0062E9D330D9D415245E24517
:108910003EDA3AD2EF20804F2A86AE866E85EA850F
:10892000EFC0BFFD5246E246EFC00F92AA842E84EC
:10893000D257125711BF97470000938727E49043FF
:10894000D443EFC03FF0E35905E419BA13075006CA
:108950006387E7001307500405456397E7EE014B73
:1089600005456FF08FD79387C1829C43945389E666
:108970009776FF1F938606706FF00FB79387C182BB
:108980009C432E86945389E69776FF1F9386866EC6
:10899000AA853E856FF04FB579714AD04ECE06D686
:1089A00022D426D2AA892E899304190003C4F4FF85
:1089B0003A8536C632C42EC23AC0EF1050402295D6
:1089C0008347150002479245A18B2246B246C9E76C
:1089D0009307D0026314F40883C70400054393048B
:1089E0002900FDC641476392E60213070003639E18
:1089F000E70083C704001307800593F7F70D63941E
:108A0000E70C83C71400C1468904B70800806314CB
:108A1000030093C8F8FF33FFD80201480145A54F72
:108A2000E54EFD5233DED802138707FD63E4EF0401
:108A3000BA8763DFD704630D58007D58636AAE00C0
:108A40006314AE006346FF0005483385A6023E95D9
:108A5000850483C7F4FFC9BF2689B9B79307B0025D
:108A60006305F400A2870143ADBF83C704009304EC
:108A70002900D5BF1387F7FB63E5EE00938797FCCA
:108A80004DBF1387F7F963E5EE00938797FA55B763
:108A9000FD57631FF8009307200223A0F9004685C5
:108AA00019EEB250225492540259F2494561828023
:108AB000630403003305A0406DD66304080093856A
:108AC000F4FF0CC2F9BF93070003A1F2A14635BF22
:108AD00013070003E38FE7F0A94605BF9387C18220
:108AE0009C43985309E71777FF1F1307A7586FF0A8
:108AF000BFEA1971A2DC86DEA6DA3284635B060067
:108B00009307B0081CC17D55F6506654D6540961D0
:108B100082803686930680202EC42ECC231AD10064
:108B2000814519C09305F4FFFD572EC82ECEBA8695
:108B30002C00231BF100AA84EF20B007FD576355DA
:108B4000F5009307B0089CC061D0A24723800700BE
:108B500065BF9387C1823687B2862E86AA858843F1
:108B60006FF03FF9011122CC26CA4AC806CE4EC684
:108B7000AA842E89328409C51C4D99E3EF10A018F0
:108B800097470000938787CC631BF406C0401C4CBA
:108B90001CC48357C400A18BD9C31C48C9C31C483B
:108BA00008409379F90F1379F90F1D8D5C486347DD
:108BB000F500A2852685EF10E00235E51C44050589
:108BC000FD171CC41C401387170018C023803701F1
:108BD0005C486389A7008357C400858B89CBA9476C
:108BE0006317F900A2852685EF00D07F0DEDF240D6
:108BF00062444A85D2444249B2490561828097471E
:108C000000009387A7C66314F400804449B79747D0
:108C100000009387A7C1E31CF4F6C0448DBFA28572
:108C2000268521202DDD7D59D9B741119387C18239
:108C300026C2844322C44AC006C62A892E8491C40F
:108C40009C4C81E72685EF10000C97470000938726
:108C5000E7BF631CF402C0400317C4009317070169
:108C6000C18393F68700BDEE93F607019DEEA547FD
:108C70002320F900136707042316E4007D55B24052
:108C80002244924402494101828097470000938721
:108C9000E7BD6314F4008044C1B797470000938791
:108CA000E7B8E31BF4FAC04445BF918B95C74C5815
:108CB00091C9930744046385F5004A85EF2040433A
:108CC000232A04028357C4002322040093F7B7FD2C
:108CD0002316F4001C481CC08357C40093E7870088
:108CE0002316F4001C4889EF8357C40013070020A3
:108CF00093F707286386E700A2854A85EF101014D2
:108D00008357C40013F7170005C75C4823240400E9
:108D1000B307F0401CCC1C480145B5F38317C400D1
:108D200013F7070829DF93E707042316F400B9B700
:108D3000898B014791E3584818C4F1BF4111194587
:108D400006C6EF2090200545EF30802C011122CC83
:108D50001C49804906CE26CA4AC84EC652C456C2CD
:108D600063C187127D141318240093894501338A47
:108D70000901130945014A9883270A0003270800BF
:108D80008507B354F7026366F706C1684E834A8EBF
:108D9000814E014FFD1811030326C3FF110E3377D7
:108DA000160141823307970233069602769793564F
:108DB0000701B3771701B307FF4036968326CEFF2E
:108DC000935E06013376160133F71601BA97C18216
:108DD00013D70741918EBA9613DF0641B3F71701F7
:108DE000C206D58F232EFEFEE3776AFA832708009A
:108DF000BDCBAA8AEF10506F634905044166850414
:108E0000CA8501457D16910903A8C9FF98419105BE
:108E1000B376C800158DB376C700AA96935707019D
:108E20001358080113D70641B3870741BA9713D5E2
:108E30000741F18EC207D58F23AEF5FEE3753AFDEB
:108E400093172400CA9798431DC72685F2406244B1
:108E5000D2444249B249224A924A0561828083271C
:108E6000080089E77D147118E36B09FF00C951B749
:108E7000984309E77D14F117E36CF9FE23A88A00F3
:108E8000E9B70145E1B775713ED85C5122C526C3EB
:108E90004AC1CEDED2DCE2D406C7D6DADAD8DED6D4
:108EA000E6D2EAD0EECE36C23AC646CAAA842E84AC
:108EB0003289C2892E8A328C89EF4145EF10300207
:108EC000C8D02322050023240500232005002326E3
:108ED0000500DC508C4389CDD84385472685B39760
:108EE000E7009CC5D8C1EF10500EDC5023A007004E
:108EF000635309048547131C190023A0F900135C70
:108F00001C00B707F07F3377FC006314F706425765
:108F10008967320C9387F770135CCC001CC3336CE9
:108F20008C00E3050C32D24791EB97470000938702
:108F3000A78F3EC039A823A00900E1B797470000DA
:108F40009387878E3EC0974700009387178E5247BE
:108F50001CC3BA402A4402459A440A49F659665A43
:108F6000D65A465BB65B265C965C065DF64D49615B
:108F70008280014681462285E28522CE62D4EFC0FE
:108F8000EFFA05E1425785471CC3973700009387E6
:108F900027773EC0D247D5DF9737000093875776B3
:108FA0007DB7B800F4006286A285268513594C016E
:108FB000EF1070751379F97FAA89A64A630D09101D
:108FC000A2577245130919C09395C700B181B7071D
:108FD000F03FDD8D02DC974700009387A780904328
:108FE000D443EFC01FDD974700009387278090434D
:108FF000D443EFC09F90973700009387A77F90439B
:10900000D443EFB07FA42A8B4A85AE8BEFD08FD4A8
:10901000973700009387877E9043D443EFC0FF8D3E
:109020002A86AE865A85DE85EFB01FA22A8BAE8BCC
:10903000EFD0CFCB2A84014681465A85DE85EFC02A
:109040007F80635B05002285EFD0CFD05A86DE8615
:10905000EFC0CFED11C17D140547D9473AD663E380
:10906000870213173400974700009387A785BA97A4
:109070009043D4437245A255EFC0CFFC6353050023
:109080007D1402D633892A41930BF9FF014B63D635
:109090000B00054B330B2B41814B634E0406A29B07
:1090A00022CC814A1247A54763E5E7149547854CD2
:1090B00063D6E7009307C7FF3EC2814C12478D4736
:1090C000630EF71063CFE704894702C8630DF70604
:1090D00085473EC88DA0364993070002569913076D
:1090E000294363D5E70213050004198D930729412D
:1090F0003315AC003354F400418DEFD0AFCCB7073B
:1091000010FEBE9585477D193EDCF1B53385E740FD
:109110003315A400DDB7330B8B40B30A804002CC7B
:1091200051B712479147630EF70005473AC81247F7
:1091300095476306F70AFD573EC4FD5DC94702C661
:1091400019A885473EC8B2476348F00A85470547D6
:109150003EC4854D3AC603A94402114723220900A3
:10916000930647018325490063FCD7082685EF1045
:10917000005DDC502320A9009C433EC0B94763E654
:10918000B71D63840C1C635E800A9377F400139709
:109190003700935C4440973700009387A772BA97D3
:1091A00093F60C0198430949DC4385C697360000C5
:1091B0009386C66E90527245D452A2553AD03ED292
:1091C000EFB09FFB0257925793FCFC002A8A2E8C2B
:1091D0000D49173D0000130D6D6C89A802C8B247F8
:1091E000A2973EC4938D1700EE87E346B0F78547FC
:1091F0009DB7854C02C2E9BDB2473EC4BE8DA1BF3A
:1092000085052322B9000607A1BF93F61C0081CE75
:1092100003260D0083264D003A85BE85EFC0EFED95
:1092200005092A87AE8793DC1C40210DE39F0CFCC7
:109230003A86BE865285E285EFB01FF42A8A2E8CCC
:1092400081A0094915CCB30C804093F7FC0013971B
:109250003700973700009387E766BA979043D44367
:109260007245A25593DC4C40173D0000130D0D6371
:10927000EFC0AFE82A8A2E8C8147639C0C12DDFF79
:10928000B25763870714173700001307A74C104322
:1092900054435285E28552D0EFC0CFDA635A0512AB
:1092A000638B0D12A2476350F00A173700001307B3
:1092B00067558257104354433E85E285EFC0EFE384
:1092C000A247130DF4FF2A8A2E8C050962874A856E
:1092D0003EDE52DABA8C3AD0EFD0CFA752580257BE
:1092E0003709C0FC4286BA86EFC02FE197360000EE
:1092F0009386C6519042D442528CEFB0EFF4F257AD
:109300002A8A2E99E1EF973700009387A750525889
:1093100002579043D4434285BA85EFC09FA9528635
:10932000CA862A8CAE8CEFC00FC7634AA054B70719
:109330000080B3C727015286BE866285E685EFC0EE
:109340006FD0634B0552724A225CB64763C7073041
:1093500039476344873013173400973700009387E9
:109360006756BA9703AB070083AB4700B24763D297
:1093700007206340B02163910D5097370000938719
:1093800067499043D4435A85DE85EFC00FD7528694
:10939000E286EFC04FC0814A01496357054A8247C0
:1093A00002470504138A1700930710032300F700F0
:1093B00045A113F71C0009CB03260D0083264D00A1
:1093C0000509EFC08FD3854793DC1C40210D75B58F
:1093D000228DEE87E5BD228D8147CDBD9386F7FFB7
:1093E00013963600973600009386C64DB296884293
:1093F000CC428246B6973EDAC247E9C397370000AF
:109400009387C7342A86AE868843CC434ADE52D03F
:10941000EFB09FD602587257173900001309893EE2
:109420004286BA86EFC0FF98024A2AD02ED2E6853D
:109430006285EFD0AF8B2ADEEFD0CF912A86AE8641
:109440006285E685EFC0FF96F2572A8CAE8C2A869D
:10945000AE8602559255050A93870703A30FFAFEBD
:10946000EFC06FB36348A00E973700009387872E35
:109470008843CC436286E686EFC0BF932A86AE86D9
:1094800002559255EFC02FB16342A018D257E30C9A
:10949000FAEA032609008326490002559255EFC0D7
:1094A000CFC503260900832649002AD02ED2628523
:1094B000E685EFC08FC42A8CAE8C95BF5286CA86D3
:1094C000EFC0AFC3525A02492AD02ED2E685628538
:1094D000EFD0CF812ADEEFD0EF872A86AE86628575
:1094E000E685EFC01F8D7257D25705091307070392
:1094F000A30FE9FE2A8CAE8C6312F906173900001F
:109500001309C924032609008326490002559255F0
:10951000EFB08FD32A86AE866285E685EFC0AFA70F
:109520006346A00E02569256032509008325490082
:10953000EFC03F882A86AE866285E685EFC08FB091
:1095400093070003E35105E00347FAFF9306FAFF90
:109550006304F7006A8459A8368AFDB7973700007C
:109560009387472A9043D443EFC02FB92A8CAE8CFF
:10957000B1BFE287BE8C8247528C973A0000938A33
:109580006A2813891700BE9D5A86DE866285E685A5
:10959000EFB09FBEEFC09FF52A8DEFC0BFFB5A868C
:1095A000DE86EFC08FB52A86AE866285E685EFC07F
:1095B0005F8093070D03A30FF9FE2A86AE864A8AC1
:1095C000639E2D07EFB04FC85A86DE862A8CAE8C7C
:1095D000EFC06F9C634BA0025A86DE866285E685EB
:1095E000EFC0CF9401E593771D0085E3CE852685F6
:1095F000EF10A01DC25723000A00050480C3D24704
:10960000E389079423A04701A9B2228D1307900391
:109610008346FAFF9307FAFF639AE6008246639D4A
:10962000F60013070003050D2380E60003C70700BB
:1096300005072380E70039BF3E8AD9BF03A60A0089
:1096400083A64A000509EFC04FAB014681462A8C2C
:10965000AE8CEFC0AF8D0DF951BF424763000710CC
:10966000924605476345D70C62579387374309E70E
:10967000264793076003998F568DDA8C854526859A
:109680003E9BBE9BEF1080372A89635E9001635C2E
:109690007001E68763D39B01DE87330BFB40B38CFD
:1096A000FC40B38BFB4063800A04C247C5CF6354C0
:1096B000A003CA856A862685EF10404A4E86AA8591
:1096C0002A892685EF1040352ACECE852685EF10D3
:1096D000C00FF247BE893386AA4111C6CE852685C2
:1096E000EF10C047AA8985452685EF102031E24753
:1096F000AA8A635BF0063E86AA852685EF1000469F
:1097000012478547AA8A014D63C8E706014D6312D7
:109710000A069317CC00528DA9EFB705F07F337C72
:10972000BC0063080C04050B850B054D99A0138D37
:10973000FDFF63CAAA01338DAA4163DE0D00B30C9D
:10974000BB41814725BFE247B30A5D41D6973ECC76
:10975000EA8A014DDDB7DA8CEE870DB7568DDA8CCB
:10976000014925B756869DBF12478547014DE3DF66
:10977000E7F8E247054589CF83A70A018D078A07E5
:10978000D697C843EF10801C930700023385A7408B
:109790005E957D8951C193070002898F1147635AF5
:1097A000F706F1473385A7402A9BAA9CAA9B6358DA
:1097B0006001CE855A862685EF102046AA89635817
:1097C0007001D6855E862685EF102045AA8AB2579D
:1097D000B1C7D6854E85EF10205163510504CE8563
:1097E000814629462685EF108002C2477D14AA894A
:1097F000638C0726CA85814629462685EF102001FD
:10980000A2472A896345F0081247894763D1E708D0
:1098100029A8E38EE7F83E85710579B76345B0075F
:109820001247894763D1E7066EC4A24791EFD685F8
:10983000814615462685EF00907DAA8AAA854E8529
:10984000EF10804AE34DA0B4B247024A13C4F7FFB9
:10985000014BD6852685EF005077E30909D86308C8
:109860000B0063062B01DA852685EF001076CA858A
:109870002685EF0090759DBB814A0149F1B76A8446
:10988000814A014929BEC2476EC46386071E6358D8
:109890009001CA8566862685EF1020382A894A8578
:1098A00063060D02832549002685EF0050690326D3
:1098B00009012A8B9305C90009060A063105EFC084
:1098C0009FE60546DA852685EF1020358247224738
:1098D0004A8B138C1700BA973EC693771A002A89D1
:1098E0003EC4D6854E85EFF06FC6DA852A8D930D7E
:1098F00005034E85EF10403F4A86AA8BD685268504
:10990000EF10A0415045930CFCFF2A8A054711E651
:10991000AA854E85EF10403D2A87D28526853AC814
:10992000EF00B06A92474247628AB3E6E700A24777
:10993000DD8E81EE130790036388ED04635470019C
:10994000930D1D032380BC0129B763CA0B00924706
:10995000B3EB7701A247B3EBFB0063950B04E35332
:10996000E0FECE8505462685EF10202BD685AA89F8
:10997000EF1080376346A00071F513F71D0079D30F
:1099800013079003E39EEDFA930790032380FC00F6
:10999000930690038347FAFF1307FAFF638CD708F7
:1099A000850745A0635BE00013079003E38EEDFCA1
:1099B00093871D002380FC0069BDB247A30FBCFF45
:1099C00063818705CE85814629462685EF00306470
:1099D000AA8981462946DA85268563182B01EF007E
:1099E00010632A8B2A89050CEDBDEF005062CA85F1
:1099F0002A8B814629462685EF0070612A89E5B7C2
:109A0000014BCE8505462685EF102021D685AA89F3
:109A1000EF10802DE34EA0F601E593F71D00ADFB9E
:109A2000930700030347FAFF9306FAFFE313F7E2F5
:109A3000368ACDBF82476399E70002470504930742
:109A400010032300F70031B53A8AA9B75247973778
:109A500000009387A7DC3EC097370000938787DC20
:109A6000631707CE6FF0EFCEA2476346F0001247B0
:109A70008947E3CCE7DA024AD6854E85EFF00FAD91
:109A80008247050A930D05033307FA40A247A30F47
:109A9000BAFFE357F7F6CE85814629462685EF00C3
:109AA0001057AA89D1BF83D7C500011122CC26CA7D
:109AB00006CE4AC84EC613F78700AA842E8479EFD3
:109AC000D841634DE000B841634AE0000145F240EF
:109AD0006244D2444249B2490561828058547DD7DC
:109AE00003A904009396370123A0040063DE060651
:109AF00070488357C400918B99C75C401D8E5C5899
:109B000099C33C401D8E5C540C508146268582973B
:109B1000FD570357C400631DF5009440F54763E902
:109B2000D706B70740208507B3D7D700858BADC3CD
:109B30001C48232204001CC09317370163D8070078
:109B4000FD576314F5009C4091E368C84C5823A06E
:109B50002401ADDD930744046385F5002685EF10ED
:109B60002059232A04029DB70C50014685462685BC
:109B70000297FD572A86E31EF5F69C40BDDB75472C
:109B80006385E70059476394E70423A024013DBFA0
:109B9000136707042316E4007D5515BF83A905014B
:109BA000E38609F203A905008D8B23A03501330953
:109BB0003941014791E3D84918C4E35920F11C54B5
:109BC0000C50CA864E86268582976349A00083572B
:109BD000C40093E707042316F4007DBFAA99330954
:109BE000A940E1BF9C49A5C3011122CC06CE2A841D
:109BF00011C51C4D81E72EC63922B24597370000AA
:109C00009387C7C4639CF5004C408397C5009DC7EC
:109C100022856244F24005616FF0FFE8973700004B
:109C20009387C7C46394F5000C44C5B79737000009
:109C30009387C7BFE39BF5FC4C44C1BFF24062442D
:109C400001450561828001458280411122C406C61A
:109C50002A842316B5002317C500232005002322DC
:109C60000500232405002322050623280500232AB6
:109C70000500232C0500214681451305C505EF602D
:109C80008FF0972700009387C7B05CD0972700001C
:109C9000938727B31CD497270000938767B75CD4BA
:109CA00097270000938727BA00D01CD8B2402244DF
:109CB0004101828097050000938505F399AA41111F
:109CC00026C2130680069384F5FFB384C4024AC0FB
:109CD0002E8922C406C693854407EF10E04B2A84E0
:109CE00001CD2320050023222501310508C4138658
:109CF00084068145EF602FE92285B24022449244D8
:109D00000249410182801C4DA5E7411106C622C4CB
:109D100097070000938747FA1CD5938781849C435B
:109D20002324050423260504232805046314F500D1
:109D300085471CCD2A84352848C022851D2808C4A3
:109D40002285052848C4484001469145EFF0FFEFC1
:109D500008440546A545EFF05FEF48440946C9456C
:109D6000EFF0BFEE85471CCCB24022444101828017
:109D7000828041119387818426C284434AC006C6EB
:109D80009C4C22C42A8981E72685EFF0DFF7938473
:109D900084048044DC40FD1763D607009C40B9CFA3
:109DA0008440C5BF0317C40039E7C1778507232264
:109DB00004062320040023220400232404005CC49E
:109DC00023280400232A0400232C04002146814573
:109DD0001305C405EF602FDB232A0402232C0402A1
:109DE00023240404232604042285B24022449244FE
:109DF0000249410182801304840671BF91454A855E
:109E0000EFF0FFEB88C049FDB1472320F900014482
:109E1000E1BF797122D44AD052CC56CA5AC85EC624
:109E200006D626D24ECE2A8AAE8A1304850401496C
:109E3000054BFD5B09ECB25022544A8592540259FD
:109E4000F249624AD24A424BB24B45618280044495
:109E500083294400FD1963D409000040E1BF83D782
:109E6000C400637BFB008397E40063877701A685CA
:109E70005285829A3369A90093848406E1BF104910
:109E80009306450113D75540B6876356C7020A06A5
:109E90000A07FD8936963697B9C913084700184353
:109EA000130300023303B3403357B700636EC80097
:109EB00098C311C391073387D740098718C96394A2
:109EC000D700232A05008280832808009107110803
:109ED000B398680033E7E80023AEE7FE0327C8FF26
:109EE000E1B711078325C7FF910723AEB7FEE36AE9
:109EF000C7FED1B7930705FD93F7F70F25476367B3
:109F0000F70001159377F50F3E8582809307F5F9E9
:109F100093F7F70F954663E5F600130595FBDDB75C
:109F20001307F5FB1377F70F8147E3EFE6FC130503
:109F300095FDC9BF1D71D6C2AA8A428536C63AC2EE
:109F400086CECAC8D2C4DAC05EDE3E8B6ED63289F7
:109F5000AE8DA2CCA6CACEC662DC66DA6AD89D25D2
:109F6000832B05005E85EFD0FFCFB387AB0083A6C0
:109F70000D0083C7F7FF7957158F3EC82A8A93874C
:109F80002600930600033306F700BE84850703C549
:109F9000F7FF32C4E309D5FEEFF0DFF5631F0510CC
:109FA0005286DE852685EF10300A631D0510338C3E
:109FB000440103450C00EFF0FFF363060510E28453
:109FC0009307000303C50400630BF500EFF09FF255
:109FD000854793391500E28C3EC4268C21A0850468
:109FE000D5B7050C03450C00EFF0DFF07DF9528684
:109FF000DE856285EF10500511E9639C0C00529CD0
:10A00000E28C03450C00EFF0FFEE5DE9014463854F
:10A010000C0033848C410A0483470C0013070005AD
:10A020006387E70013060007E28C6390C706834747
:10A030001C001307B002638BE7081307D002638B81
:10A04000E708930C1C00014D03C50C00EFF09FEADC
:10A050009307F5FF93F7F70FE14563E4F5089307DE
:10A0600005FF850C03C50C003ECAEFF0BFE8930561
:10A07000F5FF93F5F50F6148D247A948637EB80410
:10A0800063040D00B307F0403E9423A09D01638C50
:10A090000904A247814491E39944F6406644268529
:10A0A0004649D644B649264A964A064BF25B625C5C
:10A0B000D25C425DB25D256182808149814C31BFB5
:10A0C000050C81B7268C01448549B9B7014D930C25
:10A0D0002C009DBF054DE5BFB3871703AA97C11795
:10A0E00049B7E28C5DB7B3079C40FD1781451D471A
:10A0F0006344F70A5685A125054693094501B30730
:10A100004641AA8D4E8D8148814C3ECA63E984093F
:10A1100013054D0033053541098523209D0123A8F2
:10A12000AD00931455006685EF005002832B0900A3
:10A13000898C63D89B0CB3847441A6856E85EF002F
:10A1400070742A8A05C91386F4FF935656408A060E
:10A15000CE96944205473317C700758F054A19CB31
:10A160006359CA009385E4FF6E85EF00B0710D4A14
:10A1700011E1094AA6856E85EFF07FD0269403276A
:10A180008900635F8708EE85568581259247930491
:10A19000300A23A0070011B78505858791BF930773
:10A1A000FCFF3EC40346FCFFC2476309F602930767
:10A1B00000026397F80023209D018148110D814C16
:10A1C0000345FCFF46CCEFF0FFD2E2483D89224335
:10A1D00033151501B3ECAC00910815A05247930755
:10A1E000FCFF3383E700E36493FC1A855286DE8527
:10A1F00046CE1ACCEF1040656243F2484DF91A8CF6
:10A2000031B7014AE3DD74F7B3849B40EE852686BF
:10A210005685EF009020AA8D058C9309450185B7DE
:10A22000032749006355E40E3304874063457407F0
:10A230000327C9008946630AD7048D46630AD704F9
:10A240008546631BD70263998B026391EB02032758
:10A250004900B2479304200698C30547924723A8B4
:10A26000ED0023A0E90023A0B70105BD9385FBFF06
:10A270006E85EF00306161FDEE855685B92392470A
:10A280009304000523A0070009BDE3170BFEC1B727
:10A29000E31F0BFAD5B79304F4FF63180A0691C4C1
:10A2A000A6856E85EF00105E2A8A13D754400A07F0
:10A2B0004E9718438545B3959500F98D99C1136A5A
:10A2C0002A00A2856E85B38B8B40EFF05FBB032421
:10A2D00049008944630B0A080327C9008946630AB9
:10A2E000D7028D46630AD7028546631DD7001377D0
:10A2F0002A0009CB03A70900336AEA00137A1A007F
:10A30000631E0A0093E404018DA0054A79BF8544C9
:10A31000D1B70547330B6741E3060BFE83A90D0157
:10A3200013874D01FD55139A290033064701144345
:10A330006383B604850614C3894613874D0163946D
:10A34000D40883260900FD16639F760193D65B40EF
:10A350008A06369718438546B39B7601B3FBEB001C
:10A3600063830B00854493E40402924723A0B70162
:10A37000B24780C31DB31107232E07FEE369C7FA56
:10A3800003A78D0063C5E90283A54D0056858505A9
:10A390007D2603A60D019385CD002A8B09060A06AA
:10A3A0003105EFC04FB8EE8556850521DA8D03A73C
:10A3B0000D019306170011070A0723A8DD006E9709
:10A3C000854654C395BF83A60D0163DCD90085453E
:10A3D0006E85EFF0DFAA032789000504E35487F8B0
:10A3E0005DB393FBFB018544E38F0BF65297032586
:10A3F000C7FFA92B13070002B30B7741E34975FD93
:10A400009DB7A1473386C7400A0693060002918E86
:10A410005C41184111053398D70033670701B3D762
:10A42000C700232EE5FE1CC1E364B5FE82801C41FB
:10A430006548850503C6F5FF850701E61CC105458E
:10A44000828003C707009306F7FB93F6F60F636459
:10A45000D80013070702E30EC7FC014582805D7137
:10A4600052DC03AA0500A6C24EDE93545A405AD8C5
:10A470008A0486C6A2C4CAC056DA5ED662D466D240
:10A480006AD06ECE137AFA012A8BB289B294630332
:10A490000A00910483270B001389C4FF23AE04FE36
:10A4A000CA8D4A840146814A814B214C930C00029B
:10A4B0001D4D83C61700138717003AC0B1CA3685F1
:10A4C00032C63EC436C2EFF0FFA2324659E592468C
:10A4D000A24763E8DC0263D47A036378B40163467D
:10A4E000CD00EE852285EFF0DFF1214663F989008A
:10A4F000930DC4FF232E04FEDE8A6E84014682473C
:10A500004DBF93059002639CB60889072320FB008A
:10A5100063870B086379B4019D4763C6C700EE8566
:10A520002285EFF01FEE63FA8904CE87110403271A
:10A53000C4FF910723AEE7FEE37A89FE910723AEBD
:10A5400007FEE37DF9FE8327090091E763173905CC
:10A5500085472320F9001545A1A00506850B635802
:10A56000CC00E3FE89F8232E04FE054671141C403E
:10A570003D899207C98F1CC059B7E3060AFC9307AF
:10A580000002B38747417D5AB357FA0003AAC4FFBC
:10A59000337AFA0023AE44FF7DB771196DB71145C8
:10A5A000B640264496440649F259625AD25A425B52
:10A5B000B25B225C925C025DF24D61618280032598
:10A5C000C50E82801305050F82809387C1829C434C
:10A5D000885309E51765FF1F1305C5A91305050F66
:10A5E00082801971A6DAAE848395E500A2DC86DE4E
:10A5F000328463DC050083D7C40023A0060093F7F0
:10A60000070885E7930700401DA0300836C6EF1005
:10A61000C02EB246E34105FE7247BD67F98F7977D8
:10A62000BA9793B717009CC2F1BF930700041CC0F0
:10A63000F6506654D65401450961828083D7C5001F
:10A64000011122CC06CE26CA4AC8898B2E8489CF16
:10A65000930774041CC01CC885475CC8F240624460
:10A66000D24442490561828074003000AA84EFF030
:10A670005FF7A2452A892685EF00103201ED831786
:10A68000C40013F7072079FBF19B93E727002316FB
:10A69000F4007DBF97F7FFFF938707629CD4835731
:10A6A000C40008C008C893E707082316F400A247AF
:10A6B0005CC8B24791CF8315E4002685EF100027D0
:10A6C00001C98357C400F19B93E717002316F400D8
:10A6D0008357C4003369F9002316240141B79387D7
:10A6E000C182AA8588436F00302B85E141116C003F
:10A6F000014511CA795581CA834706009CC10345AB
:10A7000006003335A00041018280014519CA795500
:10A7100089CA834706009CC1034506003335A00063
:10A720008280828093F5F50F2A966314C500014557
:10A73000828083470500E38DB7FE0505FDB75C51B8
:10A74000411122C44AC006C626C22A842E8989EF36
:10A750004145EFF0DFF848D023220500232405000F
:10A7600023200500232605004450DC449DC7585093
:10A77000931729005847BA97884329E18544B39431
:10A780002401138654000A0685452285EF00F01344
:10A7900019CD2322250104C525A0130610029145D9
:10A7A0002285EF0090125C50C8C4DC47E9F30145F4
:10A7B000B24022449244024941018280184198C328
:10A7C0002328050023260500E5B75C51011122CCA2
:10A7D00006CE2A8499EF41452EC6EFF05FF0B245D0
:10A7E00048D023220500232405002320050023262A
:10A7F000050091C95450DC4113972700DC46BA97F5
:10A80000984398C18CC3F24062440561828079719B
:10A810004ECEAA89416522D426D22E84844906D6FA
:10A820004AD0D10501487D159C419105050833F7B3
:10A83000A7003307C702C183B387C7023697935671
:10A840000701698FB69793D60701C207BA9723AE5F
:10A85000F5FEE34B98FCA1C21C4463C7F4024C40D4
:10A860004E8536C68505EFF09FED10489305C40070
:10A870002A8909060A063105EFB0FFEAA2854E854E
:10A88000EFF0BFF4B2464A84938744008A07A29748
:10A89000D4C3850404C82285B2502254925402596C
:10A8A000F2494561828079719387860052CC368A5D
:10A8B000A54622D426D24ECE2E84B3C7D70206D6C2
:10A8C0004AD056CAAA89B2848546814563CCF6042B
:10A8D0004E853AC6EFF0BFE6324785471CC958C9D6
:10A8E000A54763D49704930A9400568926940509D2
:10A8F0008346F9FFAA852946938606FD4E85EFF02B
:10A900001FF1E31689FE138484FF56942689634160
:10A910004903B250225492540259F249624AD24A2F
:10A92000456182808606850555B72904A544F9BF8F
:10A93000B3079940A29783C60700AA852946938644
:10A9400006FD4E85EFF0BFEC0509D1B74177698F61
:10A95000AA87014519E3C2074145370700FF7D8FEC
:10A9600019E32105A207370700F07D8F19E31105D0
:10A970009207370700C07D8F19E309058A0763C96D
:10A98000070013971700050563440700130500022D
:10A9900082801C4113F777000DC393F6170001471F
:10A9A00099E613F7270011C785831CC105473A852F
:10A9B000828089831CC10947DDBF93960701C1824C
:10A9C000014799E2C183414793F6F70F99E22107C6
:10A9D000A18393F6F70099E21107918393F637006C
:10A9E00099E20907898393F6170081E685830507B5
:10A9F00099C31CC16DBF1307000255BF411122C48A
:10AA00002E84854506C6EFF09FD340C9B24022444C
:10AA1000054718C94101828098491C4A797126D29C
:10AA200006D622D44AD04ECEAE846354F700B28408
:10AA30002E8683A90401032906019C44CC4033845B
:10AA4000290163D38700850532C6EFF05FCF324618
:10AA500013084501131324004293C28763ED670274
:10AA600093854401939829005106131E2900C1665D
:10AA7000AE98329EFD166364C60363568000711360
:10AA800083270300F1CB00C9B250225492540259DB
:10AA9000F2494561828023A007009107C1B7832F47
:10AAA0000600B3FFDF00638A0F04428FAE82814449
:10AAB00003A7020083230F00110FB37ED700B38ECC
:10AAC000FE03B3F7D30093D303019102BE9E9357C5
:10AAD0000701B387F703A69E13D70E01B3FEDE006E
:10AAE0009E97BA9793D40701C207B3E7D701232EE5
:10AAF000FFFEE3EF12FB23209F0083522600638AB0
:10AB0000020483270800C28E2E8F814F03270F0077
:10AB100083D32E00F58F758F33075702910E110FD7
:10AB20001E977E97931F0701B3E7FF0023AEFEFE3B
:10AB30008357EFFF83AF0E004183B3875702B3FF04
:10AB4000DF00FE97BA9793DF0701E3611FFD23A0A3
:10AB5000FE001106110805B77D1405B7011126CABC
:10AB60004AC84EC606CE22CC52C4937736002A89F4
:10AB7000B284AE8989CFFD1717270000130707E1BC
:10AB80008A07BA9790438146EFF07FC8AA898984E3
:10AB9000A5CC8327490291EF4145EFF05FB4232212
:10ABA000A9022322050023240500232005002326D3
:10ABB0000500032A490203248A0019E89305102797
:10ABC0004A85EFF0BFE32324AA002A84232005004E
:10ABD00093F7140081CFCE8522864A85EFF0DFE31C
:10ABE0002A8ACE854A85EFF05FBED289858489CCDA
:10ABF000084009E92286A2854A85EFF0FFE108C0F6
:10AC0000232005002A84E9B7F24062444E85D244ED
:10AC10004249B249224A05618280797126D2AE84C6
:10AC20004ECE83A9040122D4CC41135456409C44F7
:10AC3000A2994AD056CA06D652CCAA8A13891900BC
:10AC400063C42709568532C6EFF07FAF32469307BB
:10AC500045012A8ABE8601479106634A87066353E7
:10AC60000400014494480A04338787008A069387C6
:10AC700044017D8ABE9625C2130800023308C840ED
:10AC800081458843110791073315C500C98D232ECF
:10AC9000B7FE83A5C7FFB3D50501E3E4D7FE0CC318
:10ACA00099C1138929007D1923282A015685A68573
:10ACB000EFF0BFB1B2502254528592540259F2497A
:10ACC000624AD24A456182808505860795BF23AED8
:10ACD00006FE050751B7910703A6C7FF1107232EEC
:10ACE000C7FEE3EAD7FEC1B71C499849998F8DE3A7
:10ACF0000A075105D105B306E500BA95F116F1151D
:10AD0000904298416308E600FD576363E60085477B
:10AD10003E858280E364D5FEE5BF011126CAAE847C
:10AD20004EC6B285AA89268522CC06CE4AC8328470
:10AD3000EFF09FFB05E181454E85EFF05FA0854771
:10AD40001CC9232A0500F2406244D2444249B24958
:10AD500005618280054963460500A2870149268472
:10AD6000BE844C404E85EFF09F9D0323040183A8D1
:10AD7000040113064401131E2300138844018A08AA
:10AD8000C16E23262501329EC29893064501014FCC
:10AD9000FD1E1842832F08009106B375D701B3F743
:10ADA000DF01FA959D8D93DF0F0193570701B3875C
:10ADB000F74113D70541BA9713DF0741B3F5D50122
:10ADC000C207CD8F110823AEF6FE1106E36318FD0E
:10ADD000C165FD156368C601F1169C4295C723281D
:10ADE000650095B71C429106110633F7B7007A97B4
:10ADF00013580741C183C29713DF07416D8FC20704
:10AE0000D98F23AEF6FEF9B77D13F9B7B707F07FF8
:10AE1000FD8DB707C0FCBE956355B00081473E85E8
:10AE20008280B305B04093D745414D476347F70053
:10AE3000B7050800B3D5F540D5B71387C7FEF94667
:10AE400081458547E3CDE6FCB7070080B3D7E7002F
:10AE5000F9B7797126D204494ECE930945018A0487
:10AE6000CE9422D403A4C4FF4AD02EC6228506D68F
:10AE7000EFF0DFADB24593070002898F9CC1A9476F
:10AE80001389C4FF63CDA702AD47898F3707F03F11
:10AE9000B356F400D98E014763F4290103A784FF58
:10AEA00055053315A400B357F700C98FB25022548B
:10AEB00092540259F2493E85B685456182808147A8
:10AEC00063F6290183A784FF138984FF551505C9FB
:10AED000130700023306A74033D7C7003314A4007A
:10AEE000598CB706F03FC18E014763F4290103274F
:10AEF000C9FFB397A7003357C700D98F45BFB7061F
:10AF0000F03FC18E65B7797122D42E84854526D253
:10AF10004AD0B2844ECE52CC3A8906D6368AEFF069
:10AF20001F82370710009307F7FFE58FD18093F456
:10AF3000F47FAA89B5E03EC62DC4280022C4EFF0F4
:10AF40005FA5A24621CD324793070002898FB31730
:10AF5000F700D58F3357A70023AAF9003AC6324429
:10AF600023AC890033348000050423A88900B9C4C8
:10AF70009384D4BCAA949307500323209A0033856A
:10AF8000A7402320A900B25022544E859254025962
:10AF9000F249624A45618280D98F71BF23AAD900E4
:10AFA0007DBF6800EFF0FF9EB24713050502054420
:10AFB00023AAF900854723A8F90055BF9317240059
:10AFC0001305E5BCCE972320AA00884B1604EFF0AA
:10AFD000FF97098C232089007DB779714AD02E898B
:10AFE0002C0006D622D426D24ECE52CC2A8AEFF09E
:10AFF0005FE6AA89AE842E844A856C00EFF07FE577
:10B000008327090103270A01A2461D8FB2471607AD
:10B010009D8EB307D7006355F002D2072E86338486
:10B0200097003287A2852A86BA864E85EFA0CF94F4
:10B03000B250225492540259F249624A45618280C8
:10B040003707F0FFB387E7023386B700D9BF93878E
:10B05000F5FF184A958785078A07930646010A0770
:10B06000AA97369763E5E600636AF5008280910649
:10B0700003A6C6FF1105232EC5FEEDB71105232E2D
:10B0800005FEDDB7144993D755401307450163C743
:10B09000F60263DFD700FD8981CD93962700BA962B
:10B0A00090420545B356B600B395B600631EB60090
:10B0B0008A07BA976366F70001458280B687CDBFDD
:10B0C000F1179443E5DA054582803386C502011104
:10B0D00022CC06CEB28532C6C1202A8409C53246AA
:10B0E0008145EF504FAA2285F2406244056182807B
:10B0F000DDC183A7C5FF411122C406C626C2138441
:10B10000C5FF63D307003E94AA84EF0070089387BD
:10B1100001879C4381EF2322040023A881862244D7
:10B12000B2402685924441016F00B006637EF40070
:10B1300014403307D4006396E7009843DC43369706
:10B1400018C05CC0D9BFBA87D84319C3E37DE4FEF9
:10B1500094433386D700631F86001040B29694C391
:10B160003386D700E31DC7FA10435843B29694C301
:10B17000D8C375B76375C400B1479CC04DB71040C4
:10B18000B306C4006316D70014435843B29614C0E4
:10B1900058C0C0C369B78280011126CA93843500A4
:10B1A000F19806CE22CC4AC84EC6A104B14763F33B
:10B1B000F404B14463E2B4042A89EF00607D93870C
:10B1C000018798433A8439E0938741879C4391E70C
:10B1D00081454A85CD2123AAA186A6854A85E129F4
:10B1E000FD5963193507B1472320F9004A85EF005F
:10B1F000407A29A0E3D004FCB1471CC10145F240CC
:10B200006244D2444249B249056182801C40858F24
:10B2100063CF0702AD4663F6F6001CC03E9404C03F
:10B2200031A05C406313870223A8F1864A85EF00B2
:10B2300040761305B4009307440061993307F54045
:10B240005DDF3A94898F1CC05DBF5CC3C5B72287A0
:10B25000404095BF130435007198E30285FCB305A7
:10B26000A4404A858929E31C35FBB5BF81E5B28539
:10B270006FF09FF2011122CC06CE26CA4AC84EC6F4
:10B28000328401EEEFF0DFE60149F24062444A8584
:10B29000D2444249B24905618280AE84AA89DD2D3B
:10B2A0002689E37485FEA2854E85EFF0FFEE2A899C
:10B2B00069DDA6852286EFB00FC7A6854E85EFF023
:10B2C0003FE3E1B701114AC803A9850022CC52C46B
:10B2D0005AC006CE26CA4EC656C22E84328B368A35
:10B2E00063EE260983D7C50013F7074851C704400A
:10B2F0008C495848AA8AB389B4408D44B384E40287
:10B300000947B3C4E402138716004E9763F3E400C1
:10B31000BA8493F70740D9C3A6855685EFF0DFE7D7
:10B320002A890DE5B14723A0FA008357C4007D5553
:10B3300093E707042316F400F2406244D2444249E2
:10B34000B249224A924A024B056182800C484E86DD
:10B35000EFB06FBD8357C40093F7F7B793E70708C3
:10B360002316F4002328240144C84E99B3843441A1
:10B370002320240104C4528963732A01528908409E
:10B380004A86DA85EFB08FC51C440145B387274153
:10B390001CC41C403E992320240179BF2686568573
:10B3A000EFF0DFEC2A895DFD0C485685EFF05FD4A5
:10B3B00095BF83D7C500717126D34AD14ECF06D72A
:10B3C00022D552CD56CB5AC95EC762C566C393F724
:10B3D0000708AA892E89B284B9C39C49A9E39305B9
:10B3E000000436C6EFF05FDB2320A9002328A90064
:10B3F000B24615E1B14723A0F9007D55BA502A5451
:10B400009A540A59FA496A4ADA4A4A4BBA4B2A4CC0
:10B410009A4C4D61828093070004232AF900930718
:10B420000002A30CF1029307000302DA230DF102DC
:10B4300036CE930B5002971A0000938AAA29054C26
:10B44000294B26848347040099C3639D7709B30C75
:10B450009440638E0C00E6862686CA854E85EFF002
:10B460007FE6FD576302F51AD256E69636DA834731
:10B470000400638B0718FD579304140002D002D612
:10B480003ED202D4A301010682DC83C50400154626
:10B490005685EFF02FA913841400825731E513F776
:10B4A000070109C713070002A301E10613F787008C
:10B4B00009C71307B002A301E10683C604001307FE
:10B4C000A002638BE602B2572684814625460347D5
:10B4D000040093051400130707FD6374E6068DC688
:10B4E0003ED61DA00504B9BF330555413315AC0048
:10B4F000C98F3ED0A28451BF7247930647001843BC
:10B5000036CE634907023AD6034704009307E002A8
:10B51000631FF704034714009307A002631BF7029D
:10B52000F2470904138747009C433ACE63C10702E0
:10B530003ED235A83307E04093E727003AD63ED005
:10B54000E1B7B387670385462E84BA9749B7FD579D
:10B55000C5B7050402D2814681472546034704004A
:10B5600093051400130707FD6378E606F1F283459F
:10B5700004000D461715000013054516EFF08F9ACD
:10B5800011CD97170000938767151D8D9307000451
:10B59000B397A700025505045D8D2AD083450400AA
:10B5A0001946171500001305A51393041400230C66
:10B5B000B102EFF02F9735C197B7FFFF9387276F41
:10B5C00095E70257F2471377071009CF91073ECE50
:10B5D000D257D2973EDAB5B5B387670385462E8436
:10B5E000BA97ADBF9D07E19BA107D5B7780897062D
:10B5F0000000938666CD4A860C104E85EFB0EFEAC8
:10B60000FD572A8AE316F5FC8357C9007D5593F749
:10B610000704E39507DE5255D5B378089706000076
:10B62000938686CA4A860C104E85EFB01FC5C9BFE7
:10B63000011122CC06CE2A8409C91C4D99E732C6D5
:10B640002EC4EFE04FEC3246A245971700009387D7
:10B65000E71F6316F60250401C46FD171CC663D058
:10B660000704184E63C7E70093F7F50F294763985F
:10B67000E70222856244F24005616FD0AFCE971792
:10B6800000009387A71E6314F6001044F1B79717C4
:10B6900000009387A719E311F6FC504475BF1C42C4
:10B6A00013F5F50F1387170018C22380B700F24077
:10B6B000624405618280411122C42A842E8597E765
:10B6C000FF1F23A9075A06C6EF80FFFBFD5763192A
:10B6D000F50097E7FF1F9387E7599C4391C31CC070
:10B6E000B240224441018280FD4763F6B700D9474A
:10B6F0001CC17D5582807C41011122CC06CE2E8654
:10B700002A8491C713972500BA97984319EB22858D
:10B7100032C6A528AA85228562443246F2400561D8
:10B720001DA8854601456308D700FD566319D7005B
:10B73000D9471CC00545F2406244056182802E85D0
:10B7400023A0070002970145FDB79387C182AA8510
:10B7500088436FF07FF9411122C42A842E85B28577
:10B7600097E7FF1F23A8075006C6EF007007FD5795
:10B770006319F50097E7FF1F9387C74F9C4391C359
:10B780001CC0B2402244410182806F00700341110D
:10B7900022C42E848395E50006C63924634905003A
:10B7A0007C48AA977CC8B2402244410182808357DA
:10B7B000C4007D777D17F98F2316F400EDB783D78A
:10B7C000C500011122CC26CA4AC84EC606CE93F740
:10B7D0000710AA842E843289B68991C78395E50023
:10B7E00089460146A52A8357C4007D777D17F98FC6
:10B7F0002316F4008315E4006244F240CE864A86A4
:10B80000B24942492685D244056169A0411122C44A
:10B810002E848395E50006C69122FD570357C40088
:10B82000631BF500FD77FD17F98F2316F400B24076
:10B830002244410182808567D98F2316F40068C8AD
:10B84000FDB78395E50051A005C67D160147B307F6
:10B85000E500B386E50083C7070083C6060063964C
:10B86000D7006304C7000507FDF33385D740828006
:10B870000145828091CD9307F00F63F7C7009307CE
:10B88000A0081CC17D5582802380C50005458280AB
:10B8900001458280411122C42A842E85B2853686D4
:10B8A00097E7FF1F23A8073C06C6EF80FFD9FD5787
:10B8B0006319F50097E7FF1F9387C73B9C4391C32C
:10B8C0001CC0B240224441018280411122C42A841A
:10B8D0002E8597E7FF1F23AF073806C6D125FD57F2
:10B8E0006319F50097E7FF1F9387C7389C4391C3FF
:10B8F0001CC0B240224441018280411122C42A84EA
:10B900002E85B28597E7FF1F23A6073606C64D256D
:10B91000FD576319F50097E7FF1F9387A7359C43F1
:10B9200091C31CC0B240224441018280411122C413
:10B930002A842E8597E7FF1F23AE073206C6492DBE
:10B94000FD576319F50097E7FF1F9387A7329C43C4
:10B9500091C31CC0B240224441018280411122C4E3
:10B960002A842E85B285368697E7FF1F23A40730E9
:10B9700006C6BD2DFD576319F50097E7FF1F938796
:10B98000672F9C4391C31CC0B24022444101828076
:10B990008280828083A7C5FF1385C7FF63D5070018
:10B9A000AA959C413E958280411122C42A842E850D
:10B9B000B285368697E7FF1F23AE072A06C689257C
:10B9C000FD576319F50097E7FF1F9387A72A9C434C
:10B9D00091C31CC0B24022444101828013D745016B
:10B9E000B7071000FD171347F7FF13D84601FD8D69
:10B9F000F58F931657011378F87F99CA1307F07FD4
:10BA000001456303E8008280D18F3335F0008280E6
:10BA1000C98D0545E5D5828093D74501B70610004D
:10BA20001387F6FF93F7F77F1306E03F2A886D8FA1
:10BA30000145FD816354F60099C18280828013061E
:10BA4000E0417D55E34BF6FE130530431D8D7D46E9
:10BA5000558F634AA6009387D7BE3317F700335537
:10BA6000A800598D828013053041B307F540335546
:10BA7000F7008280935746011317C60093F7F77FAC
:10BA8000797131839386170022D426D206D64AD004
:10BA90002EC83ACA02CE02CC93F6E67F2A8493548B
:10BAA000F601A1CE9166938606C0B69713D64500DF
:10BAB0009316C701C607D18E1395C5011183C5839F
:10BAC00001482316E1003247C607B7050180C58348
:10BAD000FD15C2076D8FD98F86071396F4018583F4
:10BAE000D18F48C02320040114C45CC42285B25005
:10BAF000225492540259456182803365B700A5EB08
:10BB000059CD5DC33A85EFA05FB2130715031378D3
:10BB1000F7011587631E080A100893162700B3065D
:10BB2000D6408A8813182700CC46B3870601F11641
:10BB3000CCC7E39BD8FE7D170A0732972320070066
:10BB40009306C7FF6309E6003687232007009306A4
:10BB5000C7FFE31BE6FE91679387C7C0898FC607BF
:10BB600042485245E2460357C101C58399BF15C1FA
:10BB7000A167135547009316C7013367F50013D625
:10BB800045004207D18E1395C5014183FD17014839
:10BB90000DBFA1678146FD17014701481DB78146CA
:10BBA00081470147014831BF2E852E89EFA0FFA7AD
:10BBB000130715051378F701130505021587E30D23
:10BBC00008F489476306F70009471008B14835A80B
:10BBD000B306E0408A061008B106130E0002B296C2
:10BBE00093182700330E0E4183A5C6FF9C42338372
:10BBF0001601B3D5C501B3970701DD8D2320B3002E
:10BC0000F116E313D6FE42497D171C10BE98331976
:10BC1000090123A828FF0DB793D645019397C500C6
:10BC200093F6F67FB183138616008E071357D5015E
:10BC30001376E67FFD815D8F9318350035CE13882E
:10BC400006C89307E00F63DD07018147139597004E
:10BC50009306F00FDE062581FE05558D4D8D828001
:10BC60006355000B931765000E07B337F000D98FAB
:10BC700093D8D801B3E7170113F7770063010710D2
:10BC800013F7F70091466303D700910737070004C5
:10BC90007D8F75C7130718001306F00F9376F70F03
:10BCA000E305C7FA9A07A58313959700DE06258159
:10BCB000FE05558D4D8D8280B367170199EE85CFB6
:10BCC00095479A07A5831395970093F6F60FDE061E
:10BCD0002581FE05558D4D8D8280A5DBB70740007F
:10BCE000139597009306F00FDE0681452581FE052A
:10BCF000558D4D8D82808147139597008146DE06D4
:10BD00002581FE05558D4D8D8280A5576348F80429
:10BD1000F94737068000B38707417D45598E635147
:10BD2000F504795733070741130500023357E6003E
:10BD30006388A700938626CAB316D600B3E8D80056
:10BD4000B3371001D98F13F77700014815FB13970C
:10BD500057008546E34807F48146A5B781468DB76D
:10BD6000938626C83397D8003337E000B316D60041
:10BD7000B3D8F800B367D700B3E7F800E9B7C286D5
:10BD800089B70328C500184154410C452165930724
:10BD9000F5FF13560801139E35007D8E9358D70189
:10BDA00093D7D601131308018E064111B3E7C701DB
:10BDB000B3E6160113530301131E37009308160050
:10BDC0007915F5810E033EC436C272C033F5A80062
:10BDD0001358F801B3E5650005C9717713070740EB
:10BDE0003A961307E07F635DC7041306F07F0147AF
:10BDF00081473207520631837E08518F336707012E
:10BE00003E85BA8541018280D58FCD8FB3E7C701CA
:10BE100005E2F1CB8147954693D5360013979700FD
:10BE20009396D701B3E7B60031831376F67FD1B787
:10BE3000CDDF01481306F07F37070800814755BF63
:10BE40006346C00A9307C0FC634FF60E9307D00306
:10BE50003386C7409357564037070800D98D13954E
:10BE600027000A8781462EC6B308A10011077D8AE4
:10BE7000B3E6C60163091701032E07001107B3E6F5
:10BE8000C601E31B17FF0D471D8F79CA93080101F7
:10BE9000AA9883A808FF130E0002330ECE40B39871
:10BEA000C801B3E6160175CB0A070A95B30EE10087
:10BEB0008A880C41032345009108B3D5C50033138C
:10BEC000C301B3E5650023AEB8FE1105E3931EFF81
:10BED0009145B387F540B24508082A97B3D5C50008
:10BEE0002328B7FE61A80146014721B713974600F2
:10BEF000139547003367C701F182F1839205333709
:10BF0000E000C98ECD8FD98E13F7760011C713F7D5
:10BF1000F6009145631CB702370780007D8FE30D63
:10BF200007EE05061307F07FE301E6EC370780FF15
:10BF30007D177D8F9317D7018D8226071376F67FA5
:10BF4000D58F31837DB585468147014613B7C6FF3E
:10BF500013471700BA973707800091067D8FC1B746
:10BF60008A85B388A50083A808009105050623AE3D
:10BF700015FFE358C7FE1147B307F7408A078A97B2
:10BF8000180823A007009107E39DE7FE0247B33698
:10BF9000D0009247D98E014685BF854701472DBF06
:10BFA0009307800517E7FF1F2326F7CC7D55828076
:10BFB0009307800517E7FF1F232EF7CA7D55828060
:10BFC0009307800517E7FF1F2326F7CA7D55828058
:10BFD0009307800517E7FF1F232EF7C801458280CE
:10BFE0009307800517E7FF1F2326F7C87D5582803A
:10BFF0009307800517E7FF1F232EF7C67D55828024
:10C000009307800517E7FF1F2326F7C67D5582801B
:10C0100001A0000084C400008CC4000094C400008F
:10C0200078C4000070C400009CC40000A4C40000D8
:10C0300020C20000ACC40000B4C40000BCC40000B6
:10C04000C0C4000025732573000000005379737489
:10C05000656D436C6B3A25640D0A0000322E342E58
:10C060003500000057656C636F6D6520746F205458
:10C07000656E63656E744F532074696E79282573FD
:10C08000290D0A007461736B310000007461736BD9
:10C090003200000073686F756C64206E6F742072DC
:10C0A000756E2061742068657265210D00000000C6
:10C0B0002323234920616D207461736B310D0000CF
:10C0C0007072696E740000006C65742061203D2000
:10C0D000313B000061202A3D20323B207072696EA6
:10C0E0007428277265733A272C2061293B000000D1
:10C0F000440A0000620A0000D40A0000040B000099
:10C100001E0B0000720D0000720D0000820B00007B
:10C11000720D0000720D0000CE0B0000720D0000C9
:10C12000EA0B0000720D0000720D0000720D00009D
:10C130001E0C00003A0C0000560C0000D20C00004F
:10C14000EE0C0000220D0000720D0000560D0000E4
:10C150007A120000061400004C1300003612000092
:10C160004E120000901300005A120000C813000085
:10C1700012140000F2130000DA200000E621000093
:10C18000E6210000E62100009C2000008E20000037
:10C19000E62100000222000082200000E6210000CB
:10C1A0001A200000CA1F0000F01F00002820000015
:10C1B00036200000AA200000C2200000E621000076
:10C1C0009A210000AC210000BE210000D021000017
:10C1D0006621000080210000562000003C20000065
:10C1E0006C200000241B0000301E0000461E0000D2
:10C1F000561E0000801E0000D01A00003F3F0000C5
:10C20000626164206C6873006261642063616C6CBD
:10C210000000000063616C6C696E67206E6F6E2DAC
:10C2200066756E6374696F6E0000000063616C6C0C
:10C23000206F6F6D000000006261642073747220D3
:10C240006F70000074797065206D69736D6174633F
:10C2500068000000646976206279207A65726F0058
:10C260006964656E74206578706563746564000048
:10C270006C656E67746800006C6F6F6B7570206919
:10C280006E206E6F6E2D6F626A000000756E6B6EB1
:10C290006F776E206F7020256400000070617273EC
:10C2A00065206572726F720029206578706563740D
:10C2B000656400004320737461636B0062616420F5
:10C2C000657870720000000027252E2A73272061F0
:10C2D0006C7265616479206465636C617265640089
:10C2E0004552524F523A200027252E2A7327206E9E
:10C2F0006F7420696D706C656D656E7465640000A7
:10C300006E6F7420696E206C6F6F70006E6F74209A
:10C31000696E2066756E63003B2065787065637496
:10C320006564000062616420737472206C697465D6
:10C3300072616C0027252E2A7327206E6F74206689
:10C340006F756E64000000006A732D3E62726B2090
:10C350003C3D206A732D3E73697A65002E2E2F5462
:10C36000656E63656E744F535F54696E792F746F99
:10C37000735F6A732F746F735F6A732E63000000BC
:10C380006F6F6D00286A732D3E666C61677320269F
:10C3900020465F4E4F4558454329203D3D20300003
:10C3A000627265616B000000636C61737300000072
:10C3B00063617365000000006361746368000000DE
:10C3C000636F6E7374000000636F6E74696E7565E1
:10C3D00000000000646F000064656661756C7400A5
:10C3E000656C736500000000666F720066696E61BF
:10C3F0006C6C790066616C73650000006966000012
:10C40000696E0000696E7374616E63656F6600002B
:10C410006C6574006E65770072657475726E0000ED
:10C420007377697463680000747279007468697363
:10C43000000000007468726F770000007472756508
:10C4400000000000747970656F660000766172000C
:10C45000766F6964000000007768696C6500000011
:10C4600077697468000000007969656C64000000F9
:10C470006E756C6C00000000756E646566696E65B3
:10C48000640000006F626A656374000070726F7010
:10C4900000000000737472696E6700006E756D6253
:10C4A00065720000626F6F6C65616E00636F64653A
:10C4B000726566006366756E6300000065727200E7
:10C4C0006E616E00252E3137670000002567000081
:10C4D0007B0000002C0000003A0000007D000000FE
:10C4E0002200000022635F66756E635F3078256C02
:10C4F0007822000050524F5040256C75000000001B
:10C50000565459504525640069646C65000000006C
:10C51000AA8EFFFF2E8DFFFF3E8EFFFF468EFFFF90
:10C520003E8EFFFF5E8DFFFF3E8EFFFF468EFFFFBC
:10C530002E8DFFFF2E8DFFFF5E8DFFFF468EFFFFCE
:10C54000A08EFFFFA08EFFFFA08EFFFF5E8DFFFF7E
:10C55000BA95FFFFAC94FFFFAC94FFFFAA94FFFFD6
:10C56000B294FFFFB294FFFF7894FFFFAA94FFFFFD
:10C57000B294FFFF7894FFFFB294FFFFAA94FFFFED
:10C58000A695FFFFA695FFFFA695FFFF7894FFFFF6
:10C59000000102020303030304040404040404046A
:10C5A000050505050505050505050505050505053B
:10C5B000060606060606060606060606060606061B
:10C5C000060606060606060606060606060606060B
:10C5D00007070707070707070707070707070707EB
:10C5E00007070707070707070707070707070707DB
:10C5F00007070707070707070707070707070707CB
:10C6000007070707070707070707070707070707BA
:10C61000080808080808080808080808080808089A
:10C62000080808080808080808080808080808088A
:10C63000080808080808080808080808080808087A
:10C64000080808080808080808080808080808086A
:10C65000080808080808080808080808080808085A
:10C66000080808080808080808080808080808084A
:10C67000080808080808080808080808080808083A
:10C68000080808080808080808080808080808082A
:10C690002C2066756E6374696F6E3A20000000008E
:10C6A000617373657274696F6E2022257322206630
:10C6B00061696C65643A2066696C65202225732285
:10C6C0002C206C696E65202564257325730A000093
:10C6D000232D302B20000000686C4C0065666745F8
:10C6E0004647000000000000FFFFFFFFFFFFEF7F55
:10C6F000494E4600696E66004E414E003000000013
:10C700003031323334353637383941424344454687
:10C710000000000030313233343536373839616249
:10C72000636465660000000065256C64000000001D
:10C730000000C07F16B7FFFF02B7FFFF34B7FFFF4F
:10C740003AB7FFFF16B7FFFF000000000000E03F10
:10C75000000000000000F03F00000000000000406A
:10C760000000C0FFFFFFDF419535A094FFFFDF3FD2
:10C7700035E5AF350000E03F9535A094FFFFCF3F92
:10C780006E660000696E697479000000616E0000D9
:10C7900035000000CEFBFFFFCB03000001000000CE
:10C7A0000000000034000000CEFBFFFFCB030000C0
:10C7B0000100000000000000BC89D897B2D29C3C68
:10C7C00033A7A8D523F649393DA7F444FD0FA53278
:10C7D0009D978CCF08BA5B25436FAC64280668111F
:10C7E000000000000000F83F61436F63A787D23F5D
:10C7F000B3C8608B288AC63FFB799F501344D33F50
:10C8000000000000000024400000000000001C4068
:10C810000000000000001440496E66696E6974797A
:10C82000000000004E614E0000000000000000000B
:10C8300000000000000000000000000000000000F8
:10C8400000000000000000000000000000000000E8
:10C8500000000000000000000000000000000000D8
:10C8600000000000000000000000000000000000C8
:10C8700000000000000000000000000000000000B8
:10C88000000000000000000043000000504F53492A
:10C89000580000002E0000000080E03779C34143BB
:10C8A000176E05B5B5B89346F5F93FE9034F384D16
:10C8B000321D30F94877825A3CBF737FDD4F1575C2
:10C8C000000000000000F03F0000000000002440D5
:10C8D00000000000000059400000000000408F40B0
:10C8E000000000000088C34000000000006AF8401B
:10C8F0000000000080842E4100000000D01263413F
:10C900000000000084D797410000000065CDCD41B4
:10C91000000000205FA00242000000E87648374295
:10C92000000000A2941A6D42000040E59C30A24233
:10C930000000901EC4BCD64200003426F56B0C43A8
:10C940000080E03779C3414300A0D885573476434F
:10C9500000C84E676DC1AB43003D9160E458E143B0
:10C96000408CB5781DAF154450EFE2D6E41A4B4425
:10C9700092D54D06CFF08044F64AE1C7022DB5446A
:10C98000B49DD9794378EA440500000019000000FD
:10C990007D000000002020202020202020202828AA
:10C9A000282828202020202020202020202020206F
:10C9B00020202020208810101010101010101010AF
:10C9C00010101010100404040404040404040410DF
:10C9D000101010101010414141414141010101016D
:10C9E0000101010101010101010101010101010137
:10C9F0001010101010104242424242420202020243
:10CA00000202020202020202020202020202020206
:10CA100010101010200000000000000000000000B6
:10CA20000000000000000000000000000000000006
:10CA300000000000000000000000000000000000F6
:10CA400000000000000000000000000000000000E6
:10CA500000000000000000000000000000000000D6
:10CA600000000000000000000000000000000000C6
:10CA700000000000000000000000000000000000B6
:10CA800000000000000000000000000000000000A6
:08CA900000000000000000009E
:10CA9800000000000102030401020304060708095C
:10CAA8000000000048C8000068C8000028C800004E
:10CAB800000000000000000000000000000000006E
:10CAC800000000000000000000000000000000005E
:10CAD800000000000000000000000000000000004E
:10CAE800000000000000000000000000000000003E
:10CAF800000000000000000000000000000000002E
:10CB080043000000000000000000000000000000DA
:10CB1800000000000000000000000000000000000D
:10CB280043000000000000000000000000000000BA
:10CB380000000000000000000000000000000000ED
:10CB4800430000000000000000000000000000009A
:10CB580000000000000000000000000000000000CD
:10CB6800430000000000000000000000000000007A
:10CB780000000000000000000000000000000000AD
:10CB8800430000000000000000000000000000005A
:10CB9800000000000000000000000000000000008D
:10CBA800430000000000000000000000000000003A
:10CBB800000000000000000000000000000000006D
:10CBC800430000000000000000000000000000001A
:10CBD800000000000000000000000000000000004D
:10CBE80074B80000EAA600000000000094C9000024
:10CBF80094C80000ACC00000ACC00000ACC000008D
:10CC0800ACC00000ACC00000ACC00000ACC000006C
:10CC1800ACC00000ACC00000FFFFFFFFFFFFFFFF3C
:10CC2800FFFFFFFFFFFF0000010041534349490098
:10CC380000000000000000000000000000000000EC
:10CC48000000000000000000000041534349490073
:10CC580000000000000000000000000000000000CC
:10CC680000000000000000000000000000000000BC
:10CC780000A24A0400000000E803000000000000D1
:10CC8800F0010020F0010020F8010020F801002048
:10CC9800709C002002040608749C002010000020EC
:10CCA8006C6F61646F6666006D6B73636F706500AF
:10CCB800705B00200002000010000020000000004F
:00000001FF
